:020000040000FA
:100000000C94CA010C94F2010C94F2010C94F201CC
:100010000C94F2010C94F2010C94F2010C94F20194
:100020000C94F2010C94F2010C94F2010C94F20184
:100030000C94F2010C94F2010C94F2010C94F20174
:100040000C94B1220C94F2010C947F220C9459224E
:100050000C94F2010C94F2010C94F2010C94F20154
:100060000C94FB220C94F201084AD73B3BCE016E64
:1000700084BCBFFDC12F3D6C74319ABD56833DDAFF
:100080003D00C77F11BED9E4BB4C3E916BAAAABE0E
:10009000000000803F07634236B79BD8A71A396833
:1000A0005618AEBAAB558C1D3CB7CC5763BD6DED41
:1000B000FD753EF6177231BF000000803F0800005A
:1000C00000BE922449123EABAAAA2ABECDCCCC4C8B
:1000D0003E00000080BEABAAAAAA3E00000000BFFE
:1000E000000000803F0000000000084178D3BB43BF
:1000F00087D1133D190E3CC3BD4282AD2B3E68EC47
:100100008276BED98FE1A93E4C80EFFFBE01C4FFCD
:100110007F3F0000000000004E414E494E495459B7
:10012000494E46CDCCCC3D0AD7233C17B7D13877C2
:10013000CC2B329595E6241FB14F0A0000204100D8
:1001400000C84200401C4620BCBE4CCA1B0E5AAE22
:10015000C59D7400407A10F35A00A0724E18090031
:1001600010A5D4E80000E87648170000E40B54021C
:100170000000CA9A3B000000E1F505000080969857
:1001800000000040420F000000A0860100000010A7
:100190002700000000E803000000006400000000E9
:1001A000000A00000000000100000000002C76D8CA
:1001B00088DC674F0823DFC1DFAE59E1B1B796E5B0
:1001C000E3E453C63AE651997696E8E6C28426EB14
:1001D000898C9B62ED407C6FFCEFBC9C9F40F2BA27
:1001E000A56FA5F490055A2AF75C936B6CF9676DBF
:1001F000C11BFCE0E40D47FEF520E6B500D0ED9014
:100200002E0300943577050080841E080000204EE0
:100210000A000000C80C333333330F986E12831179
:1002200041EF8D2114893BE65516CFFEE6DB18D150
:10023000844B381BF77C1D901DA4BBE42420328422
:10024000725E228100C9F124ECA1E53D27543D00F6
:10025000495220466C616D65204C6576656C3D00A9
:10026000476173206C6576656C3D0023496E76614D
:100270006C6964206B65792100204D756C7469731D
:10028000656E736F7273003E482D6669656C643AE3
:100290002028004D533D00234E6F20555620736596
:1002A0006E736F722100503D00413D0042543D008D
:1002B0004448543D00234475726174696F6E3D007B
:1002C00054494D45443D0023496E74657276616C16
:1002D0003D0054494D45493D00534156453D004779
:1002E00045540053484F57533D004C6F6767657244
:1002F000204E616D653A20004C4F474745520056ED
:10030000455253494F4E0000000000240027002AA8
:100310000000000000250028002B0023626D7020E3
:100320006661696C6564002357656C636F6D652059
:10033000746F20757365204E616E6F204C6F676718
:100340006572005245424F4F5400000000002300E8
:100350002600290004040404040404040202020226
:100360000202030303030303010204081020408078
:1003700001020408102001020408102000000008F7
:10038000000201000003040700000000000000005C
:100390001A24B82811241FBECFEFD8E0DEBFCDBF8E
:1003A00012E0A0E0B1E0E4EFF9E602C005900D92A2
:1003B000AC35B107D9F725E0ACE5B2E001C01D923C
:1003C000A630B207E1F711E0C9ECD1E004C02197F3
:1003D000FE010E94B632C83CD107C9F70E94182519
:1003E0000C94ED340C94000090910F0380910E0357
:1003F0002FEF3FEF981748F4E92FF0E0E251FD4F5F
:10040000208130E09F5F90930F03C9010895909180
:100410000F0380910E032FEF3FEF981748F4E92F59
:10042000F0E0E251FD4F208130E09F5F90930F0399
:10043000C901089591E090933C0380935E0310926C
:100440003D0310925F030895089508950895AF92B3
:10045000BF92CF92DF92EF92FF920F931F93CF93B1
:10046000DF936C017B018B01040F151FEB015E0113
:10047000AE18BF08C017D10759F06991D601ED91A8
:10048000FC910190F081E02DC6010995892B79F747
:10049000C501DF91CF911F910F91FF90EF90DF90F9
:1004A000CF90BF90AF900895FC0144815581608149
:1004B000718180E693E00C942702CF93DF930E9432
:1004C0005402EC0142E050E060E571E080E693E028
:1004D0000E9427028C0F9D1FDF91CF910895FC0190
:1004E000538D448D252F30E0842F90E0821B930B99
:1004F000541710F0CF96089501970895FC01918D3F
:10050000828D981761F0A28DAE0FBF2FB11D5D9641
:100510008C91928D9F5F9F73928F90E008958FEFE3
:100520009FEF0895FC01918D828D981731F0828D97
:10053000E80FF11D858D90E008958FEF9FEF0895EE
:10054000FC01918D228D892F90E0805C9F4F821B52
:1005500091098F739927089580E693E00E94A00285
:1005600021E0892B09F420E0822F089580E090E0BB
:10057000892B29F00E94AC0281110C94000008958F
:10058000FC01A48DA80FB92FB11DA35ABF4F2C9108
:10059000848D90E001968F739927848FA689B789FF
:1005A0002C93A089B1898C91837080648C93938DF6
:1005B000848D981306C00288F389E02D80818F7D99
:1005C00080830895EF92FF920F931F93CF93DF9351
:1005D000EC0181E0888F9B8D8C8D98131AC0E8897F
:1005E000F989808185FF15C09FB7F894EE89FF894E
:1005F0006083E889F98980818370806480839FBFEC
:1006000081E090E0DF91CF911F910F91FF90EF90EB
:100610000895F62E0B8D10E00F5F1F4F0F731127FB
:10062000E02E8C8D8E110CC00FB607FCFACFE88936
:10063000F989808185FFF5CFCE010E94C002F1CFFC
:10064000EB8DEC0FFD2FF11DE35AFF4FF0829FB7AA
:10065000F8940B8FEA89FB8980818062CFCFCF939A
:10066000DF93EC01888D8823B9F0AA89BB89E889DA
:10067000F9898C9185FD03C0808186FD0DC00FB680
:1006800007FCF7CF8C9185FFF2CF808185FFEDCFFE
:10069000CE010E94C002E9CFDF91CF91089583304F
:1006A00081F028F4813099F08230A9F008958730E4
:1006B000A9F08830C9F08430B1F4809180008F7D3A
:1006C00003C0809180008F7780938000089584B567
:1006D0008F7784BD089584B58F7DFBCF8091B00066
:1006E0008F778093B00008958091B0008F7DF9CF0F
:1006F000CF93DF93EBE8F3E08491E7E7F3E0D49165
:10070000E3E6F3E0C491CC23A1F081110E944F03F2
:10071000EC2FF0E0EE0FFF1FE65BFC4FA591B491CC
:10072000EC91ED2381E090E009F480E0DF91CF913E
:10073000089580E090E0FACF1F93CF93DF93282FA6
:1007400030E0F901E458FC4F8491F901E859FC4F7D
:10075000D491F901EC5AFC4FC491CC23A9F0162F87
:1007600081110E944F03EC2FF0E0EE0FFF1FEF5EB0
:10077000FC4FA591B4918FB7F894EC91111108C07A
:10078000D095DE23DC938FBFDF91CF911F91089529
:10079000DE2BF8CFCF93DF9390E0FC01E859FC4FBC
:1007A00024918C5A9C4FFC0184918823D1F090E0D5
:1007B000880F991FFC01E95FFC4FA591B491FC01E2
:1007C000EF5EFC4FC591D49161110EC09FB7F894B4
:1007D0008C91E22FE0958E238C932881E223E8838D
:1007E0009FBFDF91CF9108958FB7F894EC91E22BE2
:1007F000EC938FBFF6CF3FB7F8948091DA029091D7
:10080000DB02A091DC02B091DD0226B5A89B05C0F9
:100810002F3F19F00196A11DB11D3FBFBA2FA92F7F
:10082000982F8827BC01CD01620F711D811D911D7C
:1008300042E0660F771F881F991F4A95D1F70895E8
:100840008F929F92AF92BF92CF92DF92EF92FF92E0
:100850006B017C010E94FB034B015C01C114D104BC
:10086000E104F104B9F00E94FB03681979098A09CF
:100870009B09683E73408105910580F321E0C21A0F
:10088000D108E108F10888EE880E83E0981EA11CCB
:10089000B11CE4CFFF90EF90DF90CF90BF90AF906E
:1008A0009F908F9008958F929F92AF92BF92EF92F8
:1008B000FF921F93CF93DF93C82F1092FA041092E8
:1008C000FB041092FC041092FD041092FE0461E0FF
:1008D0008FE00E94CA0360E08FE00E949C036C2FAF
:1008E00070E090E080E00E94200460E08FE00E94D1
:1008F000CA038BE990E00197F1F7C0E9D1E00E94CB
:100900007803892B71F42197D1F78EEF9FEFDF9158
:10091000CF911F91FF90EF90BF90AF909F908F90DD
:100920000895C0E9D1E00E947803019719F4219756
:10093000D1F7EBCFD8E2C0E810E090E9E92EFF2430
:10094000F3940E947803892B29F481E0E81AF108D6
:10095000C1F7DBCF0E94FB034B015C0180E9E82E6D
:10096000FF24F3940E947803019729F481E0E81AA8
:10097000F108C1F7CACF0E94FB03681979098A09F7
:100980009B09693271058105910538F0E12FF0E08E
:10099000EE50FB4F80858C2B8087C69511F41F5F2E
:1009A000C0E8D15051F690E080E0B1CF8F929F9295
:1009B000AF92BF92CF92DF92EF92FF920F931F936D
:1009C000CF93DF938AE0882E912CD0E0C0E0CC2436
:1009D000CA9493E0D92EEE24EA9423E0F22EB12CAF
:1009E000A12C10E000E08091170120E4829FC0015B
:1009F0001124816080937C0080917A0080648093D0
:100A00007A0080917A0086FDFCCF909178008091E9
:100A100079008927982789270817190790F1A816C0
:100A2000B90608F45C018E159F0568F18C159D05CB
:100A300008F46C01C80FD91F65E070E080E090E019
:100A40000E94200481E0881A910869F60A0D1B1D96
:100A5000CE01801B910B8C199D098E199F0966E0B0
:100A600070E00E94A232CB01DF91CF911F910F91D4
:100A7000FF90EF90DF90CF90BF90AF909F908F90BE
:100A800008958C01D0CF7C01D5CF2FB7F894609119
:100A9000D6027091D7028091D8029091D9022FBFCF
:100AA0000895089580910E0390910F03891B990B6F
:100AB000089508952091B202260F3327331F213263
:100AC0003105ECF420913603FC0190E080E0243005
:100AD00069F082E00895A091B2022191AC014E56D6
:100AE0005D4FA40FB52FB11D2C930196861798F377
:100AF0008091B202680F6093B20280E0089581E0B5
:100B000008951092360381E080933503109210030C
:100B100061E082E10E949C0361E083E10E949C030A
:100B2000E9EBF0E080818E7F808380818D7F808300
:100B300088E48093B80085E48093BC000895109207
:100B40000F0310920E0310923D0310925F030E9458
:100B5000810584E292E09093ED028093EC0285E2BD
:100B600092E09093EB028093EA020895CF93DF9393
:100B700091E0909391028823B9F0C091B800D09190
:100B8000BA008091BC008A7B8093BC0060E082E167
:100B90000E949C0360E083E10E949C030E94810507
:100BA000D093BA00C093B800DF91CF910895CF924F
:100BB000DF92EF92FF920F931F93CF93DF93D09129
:100BC0005F0381E0D13208F09CC0C0915E030E94B7
:100BD000FB036B017C018091360381116CC082E0C4
:100BE0008093360381E0809335038FEF8093340345
:100BF00010923303D0933203AEE3B3E0E2E1F3E0CB
:100C000080E0D8138DC01092110380911103CC0F96
:100C1000C82BC093110380911003813009F084C068
:100C2000109210030E94FB036B017C018091110361
:100C30008093BB008091380390913903A0913A03CF
:100C4000B0913B03892B8A2B8B2BA1F00E94FB03D5
:100C5000009138031091390320913A0330913B03FE
:100C60006C197D098E099F09061717072807390790
:100C700008F442C08091BC0083FDD8CF85EC8093FE
:100C8000BC000E94FB036B017C0180913603823023
:100C900009F44CC0809134038F3F09F469C08091FE
:100CA0003403803209F466C080913403803309F440
:100CB00063C084E026C08091380390913903A091ED
:100CC0003A03B0913B03892B8A2B8B2B09F483CFFA
:100CD0000E94FB03009138031091390320913A03DD
:100CE00030913B036C197D098E099F090617170780
:100CF0002807390708F06FCF809137030E94B605A7
:100D000085E010923D0310925F0310923C03DF9147
:100D1000CF911F910F91FF90EF90DF90CF900895AA
:100D20009D9191938F5F6DCF85EEA9CF8091380310
:100D300090913903A0913A03B0913B03892B8A2B00
:100D40008B2B09F4A2CF0E94FB0300913803109172
:100D5000390320913A0330913B036C197D098E09C8
:100D60009F09061717072807390708F08ECFC4CF49
:100D700080E0C7CF82E0C5CF83E0C3CFCF92DF92C0
:100D8000EF92FF920F931F93CF93DF93D82FC62F2D
:100D9000613208F098C00E94FB036B017C018091D6
:100DA000360381116BC081E0809336038093350355
:100DB0009FEF90933403109233039C0F9093320370
:100DC0008093110380911103DD0FD82BD093110371
:100DD00080911003813009F078C0109210030E94B6
:100DE000FB036B017C01809111038093BB00809118
:100DF000380390913903A0913A03B0913B03892BBA
:100E00008A2B8B2BA1F00E94FB03009138031091D9
:100E1000390320913A0330913B036C197D098E0907
:100E20009F09061717072807390708F448C080915B
:100E3000BC0083FDD8CF85EC8093BC000E94FB03EF
:100E40006B017C0180913603813009F440C08091B0
:100E500033038C1710F4C0913303E2E1F3E0AEEEFC
:100E6000B2E080E08C1355C08C2FDF91CF911F91A1
:100E70000F91FF90EF90DF90CF900895809138030D
:100E800090913903A0913A03B0913B03892B8A2BAF
:100E90008B2B09F484CF0E94FB030091380310913F
:100EA000390320913A0330913B036C197D098E0977
:100EB0009F09061717072807390708F070CF809198
:100EC00037030E94B605C0E0CFCF85EEB5CF809145
:100ED000380390913903A0913A03B0913B03892BD9
:100EE0008A2B8B2B09F4AECF0E94FB0300913803B1
:100EF0001091390320913A0330913B036C197D091D
:100F00008E099F09061717072807390708F09ACF97
:100F1000D6CF91919D938F5FA5CF0895E0910F0358
:100F200080910E03E81730F4F0E0E251FD4F80812C
:100F300090E008958FEF9FEF0895CF92DF92EF92A8
:100F4000FF920F931F93CF93DF937C01CB018A0114
:100F500020913C03222389F0EB016B01C40ED51EC6
:100F6000CC15DD0569F06991D701ED91FC910190F7
:100F7000F081E02DC7010995F3CF642F0E945A0537
:100F8000C801DF91CF911F910F91FF90EF90DF90FB
:100F9000CF900895CF93DF931F92CDB7DEB76983CB
:100FA00020913C032223F9F020915F03203258F076
:100FB00021E030E0FC013383228390E080E00F9059
:100FC000DF91CF91089580913D03E82FF0E0E25C3E
:100FD000FC4F998190838F5F80933D0380935F03E3
:100FE00081E090E0ECCF61E0CE0101960E945A05CD
:100FF000F7CFCF93C82F83E50E941A026DE28DEFE1
:1010000093E00E94CA076C2F8DEF93E00E94CA07FD
:10101000CF910C94D70590E080E00895FC012481E5
:101020003581232B41F00E94540269E170E080E099
:1010300090E00C94200408950E94BE0610920F03C5
:1010400080930E030895CF93C82F87E70E941A025A
:101050006C2F8DEF93E00E94CA070E94D70587E7A7
:101060000E941A0261E070E087E790E00E941C088D
:101070000E940702C82F0E94D7058C2FCF91089598
:10108000CF93DF93C82F87E70E941A026C2F8DEF52
:1010900093E00E94CA070E94D70587E70E941A02C0
:1010A00062E070E087E790E00E941C080E9407025F
:1010B000D82F80E0C82F0E940702C82BD92B0E948E
:1010C000D705CE01DF91CF91089587E70E941A02DC
:1010D00064EF8DEF93E00E94CA076EE28DEF93E01C
:1010E0000E94CA070E94D70565E070E080E090E0AA
:1010F0000E94200486EF0C9440084F925F926F92FA
:101100007F928F929F92AF92BF92CF92DF92EF9297
:10111000FF92CF93DF9300D000D01F92CDB7DEB700
:101120000E9465084C01B12CA12C2091C704229586
:10113000220F220F207C2C5C298387E70E941A0251
:1011400064EF8DEF93E00E94CA0769818DEF93E011
:101150000E94CA070E94D7058091C704811174C1FB
:1011600065E070E080E090E00E94200486EF0E943D
:101170004008B0E0A0E0CC24D82EE92EFA2E88EF6B
:101180000E942308A7019601282B29833A834B83C9
:101190005C833091C7043D838091DC049091DD0431
:1011A000A5019401281B390B41095109A091DA04CA
:1011B000B091DB040E94B02E4B015C01AFE0B5940E
:1011C000A79497948794AA95D1F76091D4047091CD
:1011D000D504072E000C880B990BBBE0660F771F18
:1011E000881F991FBA95D1F72091D6043091D70462
:1011F000032E000C440B550B280D391D4A1D5B1D99
:101200000E94912E820E931EA41EB51E75016401CC
:1012100040EAC41A4FE0D40AE108F108A701960198
:10122000C701B6010E9492324B015C018CE0B5947B
:10123000A794979487948A95D1F7A091CC04B09104
:10124000CD040E94BB2E2B013C019DE07594679458
:10125000579447949A95D1F7A091CE04B091CF04BA
:10126000A50194010E94BB2E9C01552737FD509586
:10127000452F240D351D461D571D2E5F3F4F4F4FE7
:101280005F4F62E055954795379527956A95D1F759
:1012900030584F4F5F4FA091D804B091D9040E94AD
:1012A000B02E2B013C017FE07694679457944794CD
:1012B0007A95D1F788E090E05D81851B91092981BD
:1012C0003A814B815C8104C05695479537952795A7
:1012D0008A95D2F729833A834B835C83A091D0040B
:1012E000B091D104A50194010E94BB2E4B015C0179
:1012F000EBE0B594A79497948794EA95D1F7A091E1
:10130000CA04B091CB04A70196010E94BB2EFBE05A
:101310009595879577956795FA95D1F7680D791D1D
:101320008A1D9B1D8090C8049090C904092C000C54
:10133000AA08BB08A2E0880C991CAA1CBB1CAA9591
:10134000D1F7680D791D8A1D9B1D0D8004C0660FA5
:10135000771F881F991F0A94D2F76E5F7F4F8F4FB8
:101360009F4F24E030E040E050E00E94912E8981C0
:101370009A81AB81BC81821B930BA40BB50B9C01A2
:10138000AD0160E573EC80E090E00D8004C09695BF
:101390008795779567950A94D2F70E94923297FDC8
:1013A00066C0660F771F881F991FA30192010E94D4
:1013B000FA2E69017A019927F7FC9A958F2D7E2DD7
:1013C0006D2D9B01AC010E9492329B01AC01AEEDF0
:1013D000BBE00E94B02E4B015C01A3E4B3EEA70179
:1013E00096010E94BE2EBC01992777FD9095892F0A
:1013F0004501BB2497FCB094AB2C680D791D8A1D68
:101400009B1D6153714F8F4F9F4F44E0959587957A
:10141000779567954A95D1F76C0D7D1D8E1D9F1DA3
:101420000F900F900F900F900F90DF91CF91FF9042
:10143000EF90DF90CF90BF90AF909F908F907F9074
:101440006F905F904F900895813029F468E070E0CC
:1014500080E090E089CE823029F46EE070E080E098
:1014600090E082CE6AE170E080E090E07DCEA30162
:1014700092010E94FA2E69017A01CC0CDD1CEE1C4F
:10148000FF1C99CF0F931F93CF93DF93FC0104812F
:1014900015810115110539F4FB011082DF91CF91FF
:1014A0001F910F910895415051094017510708F4B9
:1014B0008A01EB01FC0160817181A801CE010E94CB
:1014C000C434C00FD11F1882E9CFCF93DF93C091EE
:1014D000A204D091A304209761F08991882349F058
:1014E000082E000C990B0E949E34FE0131978083D8
:1014F000F4CFDF91CF910895FC0180819181009715
:1015000011F00C94FA2860E070E0CB010895FB0123
:1015100044815581FC01248135812417350778F0F9
:1015200080819181009759F0FB0160817181611583
:10153000710529F00E94B63421E0892B09F020E0E2
:10154000822F08950F931F93CF93DF938C01EB01AC
:10155000FC01808191810097E1F0688179816115BA
:101560007105A9F0428153812C813D8142175307B7
:1015700070F00E94AF348C819D81F8019583848343
:101580001D821C82DF91CF911F910F9108950E94BF
:10159000583388819981F801918380838A819B8166
:1015A000938382838C819D819583848319821882A1
:1015B0001B821A82E5CFCF93DF93EC01888199815A
:1015C000009711F00E945833198218821D821C82E4
:1015D0001B821A82DF91CF910895FC018081918155
:1015E000009711F00C94583308950C9458330F93CE
:1015F0001F93CF93DF93EC0188819981009759F075
:101600002A813B812617370730F081E0DF91CF91A7
:101610001F910F9108958B016F5F7F4F0E94E133FF
:10162000009759F0998388831B830A832C813D811D
:10163000232B59F7FC011082E8CF80E0E7CFEF922F
:10164000FF920F931F93CF93DF936115710541F4C0
:1016500080E0DF91CF911F910F91FF90EF9008955F
:1016600041155105B1F07B01EC010C811D81040F86
:10167000151FB8010E94F70A882351F32881398188
:101680008C819D81B701820F931F0E94AF341D830F
:101690000C8381E0DECF0F931F93CF93DF9300D0B5
:1016A000CDB7DEB78C0119821A8241E050E0BE014D
:1016B0006F5F7F4F0E941F0B811103C0C8010E9402
:1016C000DB0AC8010F900F90DF91CF911F910F910E
:1016D0000895CF93DF93EC01FB0101900020E9F71F
:1016E0003197AF01461B570B0E941F0B811103C09E
:1016F000CE010E94DB0ACE01DF91CF910895CF93F6
:10170000DF93EC01FB0144815581608171810E946E
:101710001F0B811103C0CE010E94DB0ACE01DF91B5
:10172000CF910895FB0144815581608171810C94B2
:101730001F0BEF92FF920F931F93CF93DF93EC0158
:101740008B01CB010E9428297C01BC01CE010E94A3
:10175000F70A81110BC0CE010E94DB0ACE01DF9196
:10176000CF911F910F91FF90EF900895FD82EC8231
:10177000B801888199810E942129F0CFFC01118252
:10178000108213821282158214820C94990BEF92AC
:10179000FF920F931F93CF93DF93EC017B018A019C
:1017A000BA010E94F70A81110BC0CE010E94DB0A28
:1017B000CE01DF91CF911F910F91FF90EF9008958F
:1017C0001D830C83B701888199810E94AF34F0CFCB
:1017D000FB0101900020E9F73197AF01461B570B41
:1017E0000C94C70B0F931F93CF93DF93CDB7DEB746
:1017F00062970FB6F894DEBF0FBECDBF8C01CB0150
:10180000F8011182108213821282158214824AE03A
:10181000BE016F5F7F4F0E943129BE016F5F7F4F16
:10182000C8010E94E80B62960FB6F894DEBF0FBEA7
:10183000CDBFDF91CF911F910F910895CF93DF938B
:10184000EC01FB018617970749F0608171816115F2
:10185000710541F0448155810E94C70BCE01DF9193
:10186000CF9108950E94DB0AF9CFFC01118210820A
:1018700013821282158214820C941E0CFC011182B8
:1018800010821382128215821482FB0101900020C3
:10189000E9F73197AF01461B570B0C94C70BAF927A
:1018A000BF92CF92DF92EF92FF920F931F93CF934D
:1018B000DF936C015B017A0189012417350720F45D
:1018C0008F2D7901042F182F62E571E0C6010E9467
:1018D0003E0CD5011496CD91DC91EC16FD06E0F49A
:1018E0000C171D0708F4E801D501ED91FC91119743
:1018F000EC0FFD1F108110826D917C916E0D7F1D8C
:10190000C60161157105A1F00E94E80BF501808107
:101910009181C80FD91F1883C601DF91CF911F9104
:101920000F91FF90EF90DF90CF90BF90AF90089510
:101930000E94DB0AEBCFCF93DF93EC01FB01248104
:1019400035810E944F0CCE01DF91CF9108950F9306
:101950001F93CF93DF93CDB7DEB72C970FB6F894D4
:10196000DEBF0FBECDBFFC012481358112161306E8
:1019700064F48C01253131059CF40E945D0264E120
:1019800070E080E090E00E9420042C960FB6F8945E
:10199000DEBF0FBECDBFDF91CF911F910F91089594
:1019A0002FE030E050E040E0BC01CE0107960E94FD
:1019B0004F0CCE0107960E94540269E170E080E06E
:1019C00090E00E9420044FE050E0B801CE01019663
:1019D0000E949B0CBE016F5F7F4FCE0107960E9455
:1019E000A20ACE0101960E94ED0ACE0107960E943E
:1019F0005D0264E170E080E090E00E94200462E516
:101A000071E0CE0107960E94E80BCE0107960E9476
:101A1000ED0ABBCFEF92FF920F931F93CF93DF930B
:101A2000CDB7DEB7A1970FB6F894DEBF0FBECDBF1E
:101A30007C01CB01BA01F70111821082138212825C
:101A40001582148242E0420F8E010F5F1F4F0E94E9
:101A5000D828009789F0BC01C7010E94E80BA19625
:101A60000FB6F894DEBF0FBECDBFDF91CF911F91AF
:101A70000F91FF90EF900895C7010E94DB0AEFCF0E
:101A80000F931F93CF93DF938C01EB0188E2FB014F
:101A900011928A95E9F74BE050E063E571E0CE01E1
:101AA0000E94C4341B8681E090E0A0E0B0E08C8707
:101AB0009D87AE87BF87F80185899689A789B08DF4
:101AC000888B998BAA8BBB8B82E090E0A0E0B0E082
:101AD0008C8B9D8BAE8BBF8B1CA21DA21EA21FA246
:101AE00080E090E0A8E4B4E4888F998FAA8FBB8F40
:101AF00080E090E0A8E4B4EC8C8F9D8FAE8FBF8F18
:101B00008DEC9CECACE4BEE388A399A3AAA3BBA391
:101B1000DF91CF911F910F910895AF92BF92CF9215
:101B2000DF92EF92FF920F931F93CF93DF938C017D
:101B3000EB0184E2FB0111928A95E9F78EE10E94A4
:101B40001A0263E08DEF93E00E94CA070E94D70556
:101B500066E08EE10E94BE0610920F0380930E0392
:101B60008630F0F30E940702A82E0E940702B82ECA
:101B70000E940702E82E0E940702F82E0E94070228
:101B8000C82E0E940702D82E60E07A2D6B29072EFE
:101B9000000C880B990B0E945B2DF80165837683FE
:101BA0008783908760E07C2D6D29072E000C880BC1
:101BB000990B0E945B2DF801618772878387948758
:101BC00060E07E2D6F29072E000C880B990B0E9478
:101BD0005B2DF801658776878787908B118A128A3B
:101BE000138A148A84E290E0A0E0B0E088839983AD
:101BF000AA83BB8385899689A789B08D8C839D83B1
:101C0000AE83BF8382E090E0A0E0B0E08887998750
:101C1000AA87BB87188A198A1A8A1B8AC0900A0168
:101C2000D0900B01E0900C01F0900D01A7019601FE
:101C300065817681878190850E940A3020E030E0BE
:101C400048EC52E40E94BA2D6C8B7D8B8E8B9F8B5F
:101C5000A7019601F80161857285838594850E94AC
:101C60000A3020E030E048EC52E40E94BA2D688F40
:101C7000798F8A8F9B8F20910601309107014091C7
:101C8000080150910901F80165857685878590895D
:101C90000E940A3020E030E048EC52E40E94BA2D65
:101CA0006C8F7D8F8E8F9F8F81E0DF91CF911F9101
:101CB0000F91FF90EF90DF90CF90BF90AF9008957D
:101CC00085ED8093BC008091380390913903A091F9
:101CD0003A03B0913B030796A11DB11D23E0B695D1
:101CE000A795979587952A95D1F72091BC0024FD5B
:101CF00003C0109236030895409138035091390380
:101D000060913A0370913B03452B462B472B69F3B7
:101D10000097A105B10541F025E32A95F1F70000F0
:101D20000197A109B109E1CF809137030C94B60561
:101D30004F925F926F927F928F929F92AF92BF92DB
:101D4000CF92DF92EF92FF92CF93DF93CDB7DEB7C2
:101D5000CA54D1090FB6F894DEBF0FBECDBF62E5FD
:101D600071E0CE01C7960E943E0C62E571E0CE01A3
:101D7000CD960E943E0CBE016F5F7F4F8EEA94E0CD
:101D80000E948D0DCD88DE88EF88F88C20E030E051
:101D900040E251E4C701B6010E94BA2D2B013C017B
:101DA000898D9A8DAB8DBC8D2B968CAF9DAFAEAFD0
:101DB000BFAF2B9720E030E040E251E4BC01CD0101
:101DC0000E94BA2D4B015C0120E030E040E251E47A
:101DD0006D8D7E8D8F8D98A10E94BA2D27966CAF48
:101DE0007DAF8EAF9FAF2797C701B60190582B9656
:101DF0002CAD3DAD4EAD5FAD2B970E94AB2F2BEDC3
:101E00003FE049EC5FE30E942C2F209119043091B0
:101E10001A0440911B0450911C040E942C2F6B014A
:101E20007C0120E030E0A9010E94542D87FF0AC008
:101E30002BED3FE049EC50E4C701B6010E942C2F86
:101E40006B017C012BED3FE049EC50E4C701B6018A
:101E50000E94D930181654F42BED3FE049EC50E4C1
:101E6000C701B6010E942B2F6B017C0120E030E0FE
:101E700044E353E4C701B6010E94BA2D2BED3FE0C5
:101E800049E450E40E940A306B017C0120E0BC016F
:101E9000A601CE018B960E940A0D6BE571E0CE0182
:101EA00085960E943E0CBE01655D7F4FCE018596F2
:101EB0000E947F0B65E671E00E94690BBC0188EA15
:101EC00094E00E941E0CCE0185960E94ED0ACE0180
:101ED0008B960E94ED0A20E030E044EB52E4C7010B
:101EE000B6010E94542D18160CF4BFC120E030E05A
:101EF00040E05FE3C701B6010E942C2FAB01BC019B
:101F000020E0CE018B960E940A0D6CE671E0CE01B6
:101F100085960E943E0CBE01655D7F4FCE01859681
:101F20000E947F0BBC01CE01C7960E941E0CCE0101
:101F300085960E94ED0ACE018B960E94ED0A6FE60F
:101F400071E0CE01CD960E94E80B6AE671E0CE0109
:101F500085960E943E0CBE01635C7F4FCE01859644
:101F60000E947F0BBC01CE01C7960E94920BCE014E
:101F700085960E94ED0A0E944505C0905C02D090B3
:101F80005D02E0905E02F0905F026C197D098E099F
:101F90009F090E94592D20E030E04AE754E40E9456
:101FA0000A30AB01BC0123E0CE018B960E940A0DE2
:101FB0006FE771E0CE0185960E943E0CBE01655D23
:101FC0007F4FCE0185960E947F0B66E771E00E94ED
:101FD000690BBC018AE894E00E941E0CCE01859634
:101FE0000E94ED0ACE018B960E94ED0A6AE874E029
:101FF000CE0185960E94350CCE0185960E940E0872
:10200000CE0185960E94ED0A68EA74E0CE018596BD
:102010000E94350CCE0185960E940E08CE01859651
:102020000E94ED0ABE01695C7F4FCE0185960E9439
:10203000350CCE0185960E94A70CCE0185960E9494
:10204000ED0A6AE874E0CE0185960E94350C68EAD4
:1020500074E0CE0185960E947F0BBE01695C7F4FC4
:102060000E947F0BBC01CE01C7960E941E0CCE01C0
:1020700085960E94ED0A67E872E0CE0185960E947F
:10208000BE0BCE0185960E940E08CE0185960E9459
:10209000ED0A62E571E088EA94E00E94E80B21E035
:1020A000B301A201CE0185960E940A0DBE016B5DAF
:1020B0007F4F88EA94E00E94920BCE0185960E94A1
:1020C000ED0A21E027964CAD5DAD6EAD7FAD279753
:1020D000CE01C1960E940A0D21E0B501A401CE01F6
:1020E0008B960E940A0D6AE671E0CE0185960E94E9
:1020F0003E0CBE01655D7F4FCE0185960E947F0B31
:102100006AE671E00E94690BBE016F5C7F4F0E941E
:102110007F0B69E771E00E94690BBC0188EA94E0DB
:102120000E94920BCE0185960E94ED0ACE018B96FD
:102130000E94ED0ACE01C1960E94ED0A68EA74E0A1
:10214000CE0185960E94350CCE0185960E940E0820
:10215000CE0185960E94ED0AA3019201C301B2014E
:102160000E94BA2D6B017C01A5019401C501B40147
:102170000E94BA2D9B01AC01C701B6010E942C2F11
:102180006B017C0127962CAD3DAD4EAD5FAD279721
:10219000CA01B9010E94BA2D9B01AC01C701B60169
:1021A0000E942C2F0E943C316B017C016DE771E095
:1021B00088EA94E00E94E80B21E0B701A601CE0175
:1021C00085960E940A0DBE016B5D7F4FCE018B96F6
:1021D0000E94350C6AE771E0CE018B960E94690B74
:1021E000BC0188EA94E00E94920BCE018B960E947B
:1021F000ED0ACE0185960E94ED0A68EA74E0CE01F0
:1022000085960E94350CCE0185960E94A70CCE01C2
:1022100085960E94ED0A62E571E088EA94E00E94EA
:10222000E80B65E070E080E090E00E942004CE01C1
:10223000CD960E94ED0ACE01C7960E94ED0AC65BBC
:10224000DF4F0FB6F894DEBF0FBECDBFDF91CF9149
:10225000FF90EF90DF90CF90BF90AF909F908F90C6
:102260007F906F905F904F90089520E030E044E3BE
:1022700053E4C701B6010E94542D181694F0A7012B
:10228000960160E070E884E393E40E942B2FAB0199
:10229000BC0120E0CE018B960E940A0D61E771E03F
:1022A00036CE20E030E047E853E4C701B6010E9493
:1022B000542D181694F120E030E044E353E4C701B4
:1022C000B6010E942B2F20E030E040E05FE30E9447
:1022D0002C2FAB01BC0120E0CE018B960E940A0D91
:1022E00061E771E0CE0185960E943E0CBE01655DFE
:1022F0007F4FCE0185960E947F0BBC01CE01C79611
:102300000E941E0CCE0185960E94ED0ACE018B968E
:102310000E94ED0A64E771E014CEA701960160E027
:1023200070E084EB93E40E942B2F20E030E040E04B
:102330005FE30E942C2F0E947C30CE018B960E947E
:10234000F20B6CE671E0CECFFF920F931F93CF9309
:10235000DF93EC01F62E08811981C8010E947B2EC3
:10236000F81621F06F2DC8010E94832ECE01DF9157
:10237000CF911F910F91FF900895EF92FF920F93CD
:102380001F93CF93DF9300D0CDB7DEB709E014E001
:10239000895094407C01C701800F911F9A838983E3
:1023A000F80161918F01CE0101960E94A411F4E021
:1023B00007351F0781F789E094E00F900F90DF91B8
:1023C000CF911F910F91FF90EF900895EF92FF92A0
:1023D0000F931F93CF93DF9300D0CDB7DEB707E500
:1023E00014E0875594407C01C701800F911F9A83A8
:1023F0008983F80161918F01CE0101960E94A41199
:10240000F4E00E371F0781F787E594E00F900F90F7
:10241000DF91CF911F910F91FF90EF9008952F9230
:102420003F924F925F926F927F928F929F92AF9264
:10243000BF92CF92DF92EF92FF920F931F93CF93B1
:10244000DF93CDB7DEB76E970FB6F894DEBF0FBE41
:10245000CDBF6FEF72E0CE0101960E94BE0BBE01B0
:102460006F5F7F4F82EA94E00E94870A182FCE01A7
:1024700001960E94ED0A112399F161E871E0CE0105
:1024800001960E943E0C6EE774E0CE0101960E9418
:102490007F0BBC0188EA94E00E941E0CCE010196DD
:1024A0000E94ED0A6BE871E0CE0107960E943E0C97
:1024B00068EA74E0CE0107960E947F0BBC01CE0152
:1024C00001960E94350CCE0101960E94A70CCE0108
:1024D00001960E94ED0ACE0107960E94ED0A52C0B5
:1024E00068EF72E0CE0101960E94BE0BBE016F5FE5
:1024F0007F4F82EA94E00E94870A182FCE0101964E
:102500000E94ED0A112369F06AEE72E088EA94E015
:102510000E94990B64E874E088EA94E00E94920BB0
:10252000C1CF63EE72E0CE0101960E94BE0BBE01E8
:102530006F5F7F4F82EA94E00E94870A182FCE01D6
:1025400001960E94ED0A1123D9F127E030E046E020
:1025500050E066E974E0CE0101960E944F0CBE0186
:102560006F5F7F4F80E994E00E94A20ACE0101963E
:102570000E94ED0A80E994E00E947C0A672B21F416
:102580001092E00281E003C081E08093E0026E9649
:102590000FB6F894DEBF0FBECDBFDF91CF911F9174
:1025A0000F91FF90EF90DF90CF90BF90AF909F90F2
:1025B0008F907F906F905F904F903F902F900895F5
:1025C0006FED72E0CE0101960E94BE0BBE016F5FFF
:1025D0007F4F82EA94E00E94870A182FCE0101966D
:1025E0000E94ED0A112309F4BAC080918F029091E4
:1025F00090021816190634F688EC90E090930501C5
:102600008093040180E693E00E942F031D861E86BE
:102610001F86188ACC24C394D12C40EC242E43E08E
:10262000342E5E012DE0A20EB11C2E0131E1430ECD
:10263000511C5FE8652E52E0752E80918F029091BB
:1026400090028C159D050CF49DCF80910401909112
:102650000501813C934024F0309205012092040151
:102660000091040110910501750148018A189B0829
:10267000C4018E0D9F1D0E947B2EF70181937F0167
:102680004E165F06A9F7C801049690930501809342
:1026900004012BE6E22E22E0F22E07561240C8017A
:1026A0008E0D9F1D0E947B2EF70181937F016E1678
:1026B0007F06A9F74D855E856F85788923E0CE0179
:1026C00007960E940A0DBE01695F7F4FCE010196F9
:1026D0000E94350C66E771E0CE0101960E94690BFD
:1026E000BC0188EA94E00E941E0CCE0101960E9473
:1026F000ED0ACE0107960E94ED0A6BE672E0CE016C
:1027000001960E943E0CBE016F5F7F4F88EA94E005
:102710000E94920BCE0101960E94ED0A68EA74E0D5
:10272000CE0101960E94350CCE0101960E94A70CA5
:10273000CE0101960E94ED0A80910401909105015D
:102740008496909305018093040164E170E080E039
:1027500090E00E942004FFEFCF1ADF0A6ECF69EDF0
:1027600072E0CE0101960E94BE0BBE016F5F7F4FEB
:1027700082EA94E00E94870A182FCE0101960E94F7
:10278000ED0A1123F1F126E030E045E050E066E982
:1027900074E0CE0101960E944F0CBE016F5F7F4F27
:1027A00080E994E00E94A20ACE0101960E94ED0AFF
:1027B00080E994E00E947C0A672B19F410926A0267
:1027C000E1CE81E080936A0288EC90E0909305016D
:1027D000809304011092900210928F021092660270
:1027E0001092670210926802109269020E944505D9
:1027F0006093620270936302809364029093650217
:10280000C1CE62ED72E0CE0101960E94BE0BBE0108
:102810006F5F7F4F82EA94E00E94870A182FCE01F3
:1028200001960E94ED0A112309F47FC080919A0459
:1028300090919B04079708F4A5CE46E050E066E926
:1028400074E0CE0101960E949B0CBE016F5F7F4F2A
:1028500080E994E00E94A20ACE0101960E94ED0A4E
:102860008091900490919104009709F45AC00E94BD
:10287000F6286093130170931401809315019093CF
:10288000160167EC72E088EA94E00E94990B40918F
:10289000130150911401609115017091160122E00D
:1028A000CE0107960E940A0DBE01695F7F4FCE01DF
:1028B00001960E94350C6DE871E0CE0101960E94F0
:1028C000690BBC0188EA94E00E94920BCE0101964C
:1028D0000E94ED0ACE0107960E94ED0A68EA74E0B4
:1028E000CE0101960E94350CCE0101960E94A70CE4
:1028F000CE0101960E94ED0A0E94450528EE33E0C4
:1029000040E050E00E94FA2ECA01B9010E94592D00
:102910006093E5027093E6028093E7029093E802E9
:1029200031CE60E070E0CB01A4CF60EC72E0CE016C
:1029300001960E94BE0BBE016F5F7F4F82EA94E05A
:102940000E94870A182FCE0101960E94ED0A1123DA
:1029500009F469C080919A0490919B04079708F448
:1029600011CE46E050E066E974E0CE0101960E9487
:102970009B0CBE016F5F7F4F80E994E00E94A20A2A
:10298000CE0101960E94ED0A8091900490919104ED
:10299000009709F444C00E94F628609300017093E8
:1029A0000101809302019093030165EB72E088EAD4
:1029B00094E00E94990B40910001509101016091B7
:1029C00002017091030121E0CE0107960E940A0DD9
:1029D000BE01695F7F4FCE0101960E94350C6DE804
:1029E00071E0CE0101960E94690BBC0188EA94E077
:1029F0000E94920BCE0101960E94ED0ACE0107962D
:102A00000E94ED0A68EA74E0CE0101960E94350C3E
:102A1000CE0101960E94A70CCE010196AFC160E0E5
:102A200070E0CB01BACF60EB72E0CE0101960E945C
:102A3000BE0BBE016F5F7F4F82EA94E00E94870A5F
:102A4000182FCE0101960E94ED0A112341F126E0D4
:102A500030E044E050E066E974E0CE0101960E9467
:102A60004F0CBE016F5F7F4F80E994E00E94A20A85
:102A7000CE0101960E94ED0A80E994E00E947C0A52
:102A800070930A04609309047093100160930F011E
:102A900080911101909112010E94BD1173CD6CEAD9
:102AA00072E0CE0101960E94BE0BBE016F5F7F4FA8
:102AB00082EA94E00E94870A182FCE0101960E94B4
:102AC000ED0A1123A9F143E050E066E974E0CE017C
:102AD00001960E949B0CBE016F5F7F4F80E994E0DE
:102AE0000E94A20ACE0101960E94ED0A60E974E0FC
:102AF000CE0101960E94350CCE0101960E944B0B2F
:102B0000BC0184E894E00E941E0CCE0101960E9454
:102B1000ED0A40918804509189044115510509F44A
:102B2000B7CF6BE074E084E894E00E94420AB0CF33
:102B300069EA72E0CE0101960E94BE0BBE016F5F92
:102B40007F4F82EA94E00E94870A182FCE010196F7
:102B50000E94ED0A112321F142E050E066E974E0A1
:102B6000CE0101960E949B0CBE016F5F7F4F80E9F2
:102B700094E00E94A20ACE0101960E94ED0A80E92B
:102B800094E00E947C0A709361026093600263305B
:102B9000710508F4F7CC1092610210926002F2CC39
:102BA00066EA72E0CE0101960E94BE0BBE016F5F25
:102BB0007F4F82EA94E00E94870A182FCE01019687
:102BC0000E94ED0A112309F48DC080919A0490911E
:102BD0009B04409708F0CEC242E050E066E974E002
:102BE000CE0101960E949B0CBE016F5F7F4F80E972
:102BF00094E00E94A20ACE0101960E94ED0A809103
:102C00009004909191040097A9F10E94F62820E089
:102C100030E048EC52E40E94BA2D0E947C30609370
:102C200015047093160480931704909318048B0175
:102C30009C0100591F452140310901341C492105DF
:102C40003105E0F06FE871E0CE0101960E943E0C84
:102C500060E974E0CE0101960E947F0B65E971E0A6
:102C60000E94690BBC0188EA94E00E941E0CCE0110
:102C7000019633CC60E070E0CB01C9CF0E945B2DA0
:102C800020E030E048EC52E40E940A30AB01BC0185
:102C900022E0CE0101960E940A0DBE016F5F7F4FB8
:102CA00088EA94E00E94A20ACE0101960E94ED0AF1
:102CB00065EA71E0CE0101960E943E0C68EA74E07C
:102CC000CE0101960E947F0B62EB71E00E94690BBE
:102CD000BC0188EA94E00E941E0CCE0101960E947D
:102CE000ED0AD6CE67EB71E0CE0101960E943E0C54
:102CF000BE016F5F7F4F82EA94E00E94870A182F1F
:102D0000CE0101960E94ED0A1123D9F1809155045C
:102D100090915604019709F035CC62E571E0CE013F
:102D20000D960E943E0C89899A89009729F1ED85BC
:102D3000FE852081222301F10797F0F06DEB71E011
:102D4000CE0107960E943E0CBE01635F7F4FCE010D
:102D500007960E947F0BBC01CE0101960E94350CA4
:102D6000CE0101960E94A70CCE0101960E94ED0AA9
:102D7000CE0107960E94ED0ACE010D960E94ED0A43
:102D800001CC6BEC71E0CE0101960E943E0CBE01BD
:102D90006F5F7F4F82EA94E00E94870A182FCE016E
:102DA00001960E94ED0A1123F1F025E030E044E0A5
:102DB00050E066E974E0CE0101960E944F0CBE011E
:102DC0006F5F7F4F80E994E00E94A20ACE010196D6
:102DD0000E94ED0A80E994E00E947C0A70935604F8
:102DE0006093550455CE60ED71E0CE0101960E94CE
:102DF0003E0CBE016F5F7F4F82EA94E00E94870A1B
:102E0000182FCE0101960E94ED0A112339F067E9CF
:102E100072E088EA94E00E94990BF4CD63E972E0D5
:102E2000CE0101960E94BE0BBE016F5F7F4F82EA0A
:102E300094E00E94870A182FCE0101960E94ED0AA5
:102E4000112309F49FCB43E050E062EA74E0CE0125
:102E500007960E949B0CBE01695F7F4FCE010196D1
:102E60000E94350CCE0101960E944B0BBC0180E9FB
:102E700094E00E941E0CCE0101960E94ED0ACE0144
:102E800007960E94ED0A60E974E0CE0149960E941F
:102E9000350C64ED71E0CE0101960E943E0C8D8DE3
:102EA0009E8D892BC9F1098D1A8D69817A81C8019E
:102EB0000E94D334009781F1FC01E01BF10B8F01DC
:102EC000CE0101960E94ED0A62E571E0CE014396C3
:102ED0000E943E0C62E571E0CE010D960E943E0C10
:102EE00010161106E4F466ED71E0CE0101960E9421
:102EF0003E0CCE0101960E94A70CCE0101960E94C5
:102F0000ED0ACE010D960E94ED0ACE0143960E9475
:102F1000ED0ACE01499632CF0FEF1FEFD1CFBE01A0
:102F2000675E7F4FCE010D960E941E0CD12CC12CE6
:102F30008AEF682E77247A9496E0592E89899A89A7
:102F4000009709F408C1F5E0CF16D104C9F36BEB83
:102F500071E0CE0101960E943E0CBE016F5F7F4F73
:102F6000CE010D960E94870A182FCE0101960E946D
:102F7000ED0A1111C9C001E010E0980150E040E0F5
:102F8000BE01635F7F4FCE0107960E944F0CBE01CA
:102F9000695F7F4FCE0101960E94350CCE010196EC
:102FA0000E944B0BBC01CE0143960E941E0CCE0129
:102FB00001960E94ED0ACE0107960E94ED0ABE011D
:102FC0006D5E7F4FCE0107960E94350C8B859C85E8
:102FD000029708F49CC06BEB71E0CE0101960E9451
:102FE0003E0CBE016F5F7F4FCE0107960E94870A9D
:102FF000F82ECE0101960E94ED0AFF2009F487C049
:1030000022E030E041E050E0BE01695F7F4FCE0139
:1030100001960E944F0CCE0101960E947C0A4B0142
:103020007B01CE0101960E94ED0A97FE03C02CE1C0
:10303000E20EF11CB3016E197F095C9C70015D9C6E
:10304000F00C1124F701E95AFB4F76876587CE0112
:1030500007960E94ED0AB701605A7B4F44E050E0AA
:10306000CE0143960E94420A3FEFC31AD30A8989D0
:103070009A890817190708F067C0A801BE01635FA5
:103080007F4FCE0101960E949B0CBE016F5F7F4F68
:10309000CE0143960E94A20ACE0101960E94ED0A3B
:1030A000BE016D5E7F4FCE010D960E941E0CAD8459
:1030B000BE84A114B10409F441CF09891A897501AC
:1030C0000115110509F43ACF47014FEF841A940A0C
:1030D000F7018081082E000C990B0E94232D892B6B
:1030E000D9F4015011090A0D1B1DF8018081082E29
:1030F000000C990B0E94232D892B81F00E151F05C2
:1031000068F001501109F1CF02E010E036CFCE0196
:1031100007960E947C0A91CF7401D6CF0F5F1F4F94
:10312000A8014E195F095A8B498BAE14BF0420F4D5
:10313000B701C5010E94A634ED85FE8589899A896B
:10314000E80FF91F1082FACE62E571E0CE010D960C
:103150000E94E80BF3CEC0925904CC2041F081E0EC
:10316000809357048EE190E00E94E611CACE10923F
:103170005704F8CF80E00BCA8F929F92AF92BF9214
:10318000CF92DF92EF92FF920F931F93CF93DF9333
:1031900000D000D000D0CDB7DEB720916A02222344
:1031A00009F4A4C020918F0230919002243131059E
:1031B0000CF09CC00091040110910501013C43E01A
:1031C00014070CF093C06C012F5F3F4F30939002B7
:1031D00020938F020E9445058090620290906302C6
:1031E000A0906402B0906502681979098A099B0968
:1031F0000E94592D20E030E04AE754E40E940A3052
:1032000060936602709367028093680290936902EC
:10321000083C110534F488EC90E09093050180930C
:103220000401809104019091050106E612E0FC0181
:10323000E656F2407F01C701800F911F9A83898370
:10324000F80161918F01CE0101960E94A411F2E074
:103250000A361F0781F7E0900401F0900501C701CD
:1032600004969093050180930401B601CE01019666
:103270000E94350CCE0101960E944B0BBC0188EADE
:1032800094E00E941E0CCE0101960E94ED0A40912E
:10329000AC045091AD044115510531F06BE672E07C
:1032A00088EA94E00E94420A8FE8C82E82E0D82E75
:1032B0000BE612E09701275632407901C701800FD3
:1032C000911F9A838983F80161918F01CE01019644
:1032D0000E94A411C016D10689F780910401909133
:1032E00005018496909305018093040126960FB6FC
:1032F000F894DEBF0FBECDBFDF91CF911F910F912C
:10330000FF90EF90DF90CF90BF90AF909F908F9005
:1033100008952F923F924F925F926F927F928F9279
:103320009F92AF92BF92CF92DF92EF92FF920F9354
:103330001F93CF93DF93CDB7DEB7CC55D1090FB62E
:10334000F894DEBF0FBECDBF29966CAF7DAF8EAFB8
:103350009FAF299725962CAF3DAF4EAF5FAF259716
:10336000683E73408105910554F088E290E0A0E04A
:10337000B0E029968CAF9DAFAEAFBFAF2997259631
:103380002CAD3DAD4EAD5FAD25972115314E454F6E
:10339000554054F020E031EE45EF55E025962CAF36
:1033A0003DAF4EAF5FAF25978091E902882351F082
:1033B00081E090E0A0E0B0E025968CAF9DAFAEAF8D
:1033C000BFAF25970E94450569966CAF7DAF8EAF64
:1033D0009FAF69970E9445052D966CAF7DAF8EAF6C
:1033E0009FAF2D9769966CAD7DAD8EAD9FAD699702
:1033F00028EE33E040E050E00E94912E6D962CAF15
:103400003DAF4EAF5FAF6D9711E001E01E0197E059
:10341000290E311C2D966CAD7DAD8EAD9FAD2D97D7
:1034200069962CAD3DAD4EAD5FAD6997621B730BD8
:10343000840B950B25962CAD3DAD4EAD5FAD25971C
:1034400062177307840795070CF03BC30E945B2D3E
:1034500020E030E04AE754E40E940A30AB01BC01AE
:1034600023E0CE0101960E940A0DBE016F5F7F4FDF
:1034700080E994E00E94A20ACE0101960E94ED0A22
:1034800025968CAD9DADAEADBFAD25970A97A10534
:10349000B10524F518AA1FA61AAA19AA1CAA1BAAC4
:1034A0002AE0AE014F5F5F4F6D966CAD7DAD8EAD86
:1034B0009FAD6D970E943C29BE016F5F7F4FCE018B
:1034C0008F960E94E80BBE01615D7F4F80E994E01A
:1034D0000E94A20ACE018F960E94ED0A8091E90215
:1034E000882371F162E571E080E994E00E94E80BC5
:1034F00083E50E941A0262E38DEF93E00E94CA07FF
:103500000E94D70583E50E941A0266E070E083E519
:1035100090E00E941C082EEDE22E24E0F22EC7015E
:103520008E5D9440AFEFEA1AFA0A30910E032091B3
:103530000F033217F9F00E940702F7018587EFCFDA
:103540006FE771E0CE0101960E943E0C60E974E0E5
:10355000CE0101960E947F0B66E771E00E94690B25
:10356000BC0180E994E00E941E0CCE0101960E94ED
:10357000ED0ABECF069721F01092DE040093DF041F
:103580000E94D7058091EC049091ED049A83898381
:103590008091EE049091EF049C838B838091F004E2
:1035A0009091F1049E838D839E012F5F3F4F79019F
:1035B00090EE492E94E0592E3E0133E2630E711CC9
:1035C0006301D7016D917D917D01F2018190919010
:1035D000A190B1902F01072E000C880B990B0E942F
:1035E0005B2DA50194010E94BA2DD6016D937D93A8
:1035F0008D939D936D012E143F0419F762E571E0E0
:1036000088EA94E00E94E80B2301BCE04B0E511CB9
:10361000C12CD12C7601F30181909190A190B190B1
:103620003F01A5019401C501B4010E94BA2D9B017F
:10363000AC01C701B6010E942C2F6B017C0123E075
:10364000B501A401CE0101960E940A0DBE016F5F73
:103650007F4FCE018F960E94350C6AE671E0CE0155
:103660008F960E94690BBC0188EA94E00E94920B3D
:10367000CE018F960E94ED0ACE0101960E94ED0ABE
:103680006414750441F6C701B6010E943C316B0118
:103690007C012DEC3CEC4CE45FE30E94D930181621
:1036A0000CF071C12AE939E949E95FE3C701B601C4
:1036B0000E94542D880F880B1823809160029091EE
:1036C00061028130910509F473C1029719F0112349
:1036D00009F46EC18BA49CA4ADA4BEA44BA05CA0B5
:1036E0006DA07EA0CFA0D8A4E9A4FAA420E030E089
:1036F000A901C501B4010E94542D882309F445C1D4
:10370000A3019201C301B2010E94BA2D61966CAF70
:103710007DAF8EAF9FAF6197A7019601C701B6013C
:103720000E94BA2D9B01AC0161966CAD7DAD8EAD52
:103730009FAD61970E942C2F0E943C31A5019401FE
:103740000E94AB2F20EE3EE245E652E40E94BA2DE5
:1037500061966CAF7DAF8EAF9FAF619720E030E098
:10376000A901C701B6010E94542D882309F412C192
:10377000A3019201C301B2010E94BA2D65966CAFFC
:103780007DAF8EAF9FAF6597A5019401C501B401D0
:103790000E94BA2D9B01AC0165966CAD7DAD8EADDE
:1037A0009FAD65970E942C2F0E943C31A701960186
:1037B0000E94AB2F20EE3EE245E652E40E94BA2D75
:1037C00065966CAF7DAF8EAF9FAF659720E030E020
:1037D000A901C301B2010E94542D882309F4DFC05E
:1037E000A5019401C501B4010E94BA2D4B015C01F1
:1037F000A7019601C701B6010E94BA2D9B01AC0139
:10380000C501B4010E942C2F0E943C31A3019201FA
:103810000E94AB2F6B017C0160E974E0CE01019640
:103820000E94350C6DEE71E0CE0101960E94690B8D
:10383000BC0188EA94E00E941E0CCE0101960E9411
:10384000ED0A68EA74E0CE0101960E94350CCE01C3
:1038500001960E940E08CE0101960E94ED0A21E019
:1038600061964CAD5DAD6EAD7FAD6197CE01CB96EF
:103870000E940A0D21E065964CAD5DAD6EAD7FAD49
:103880006597CE01C5960E940A0D20EE3EE245E600
:1038900052E4C701B6010E94BA2DAB01BC0121E080
:1038A000CE0101960E940A0DBE016F5F7F4FCE01CF
:1038B0008F960E94350C6AE671E0CE018F960E94C9
:1038C000690BBE016B5C7F4F0E947F0B6AE671E063
:1038D0000E94690BBE01655C7F4F0E947F0BBC019B
:1038E00088EA94E00E941E0CCE018F960E94ED0A99
:1038F000CE0101960E94ED0ACE01C5960E94ED0A06
:10390000CE01CB960E94ED0A68EA74E0CE010196E2
:103910000E94350CCE0101960E94A70CCE010196A3
:103920000E94ED0A11E00E944505DC01CB012D96B5
:103930002CAD3DAD4EAD5FAD2D97821B930BA40B0F
:10394000B50B29962CAD3DAD4EAD5FAD29978217D5
:103950009307A407B50744F4281B390B4A0B5B0BEC
:10396000CA01B9010E9420040E9445052D966CAF42
:103970007DAF8EAF9FAF2D9762E571E088EA94E04E
:103980000E94E80B47CD10E098CE6BED7FE089EC0C
:103990009FE3D8CE6BED7FE089EC9FE30BCF8BEDFF
:1039A000C82E8FE0D82E89ECE82E8FE3F82E34CF86
:1039B00065E072E0CE0101960E943E0C68EA74E078
:1039C000CE0101960E947F0BBC0188EA94E00E9420
:1039D0001E0CCE0101960E94ED0A68EA74E0CE0149
:1039E00001960E94350CCE0101960E94A70CCE01D3
:1039F00001960E94ED0A68EA74E0CE0101960E94E9
:103A0000350CCE0101960E94BC18CE0101960E9491
:103A1000ED0A23E0B701A601CE018F960E940A0DA0
:103A200062E172E0CE0101960E943E0CBE01615D32
:103A30007F4FCE0101960E947F0B65E172E00E94EC
:103A4000690BBC0188EA94E00E941E0CCE0101962D
:103A50000E94ED0ACE018F960E94ED0A68EA74E09A
:103A6000CE0101960E94350CCE0101960E94BC1831
:103A7000CE0101960E94ED0A60E974E0CE01019644
:103A80000E94350C68EA74E0CE0101960E947F0B1B
:103A9000BC0188EA94E00E941E0CCE0101960E94AF
:103AA000ED0A68EA74E0CE0101960E94350CCE0161
:103AB00001960E94A70CCE0101960E94ED0A10E02B
:103AC00032CFC45ADF4F0FB6F894DEBF0FBECDBF62
:103AD000DF91CF911F910F91FF90EF90DF90CF90EA
:103AE000BF90AF909F908F907F906F905F904F901E
:103AF0003F902F9008954F925F926F927F928F9296
:103B00009F92AF92BF92CF92DF92EF92FF920F936C
:103B10001F93CF93DF93CDB7DEB72C970FB6F894F2
:103B2000DEBF0FBECDBF7C0162E571E088EA94E0A4
:103B30000E94E80BC7010596059768F08091E9029D
:103B4000811109C02CEEE2162FEFF20624F0F0925C
:103B5000E402E092E302F7017A96E432F10508F01C
:103B60007DC4EB54F24E0C94B632BB212E22B72109
:103B70002E222E222E222E222E222E222E222E22C5
:103B8000DB1DDB1DDB1DDB1DDB1DDB1DDB1DD91D77
:103B9000DB1DDB1D1A1E291E2C1E2E22DB1DDB1D2C
:103BA0003A1EB11FDB1DD820F6200021DB1DDB1DD6
:103BB0007E210E9445058091AC049091AD04892B33
:103BC000E1F068EA74E0CE0101960E94350CCE0166
:103BD00001960E94A70CCE0101960E94ED0A68EAA8
:103BE00074E0CE0101960E94350CCE0101960E9430
:103BF000BC18CE0101960E94ED0A64E670E080E0F8
:103C000090E00E9420042C960FB6F894DEBF0FBE01
:103C1000CDBFDF91CF911F910F91FF90EF90DF907B
:103C2000CF90BF90AF909F908F907F906F905F905C
:103C30004F9008958091E902882321F088EA94E06A
:103C40000E945D0268EC70E080E090E00E94200439
:103C5000B2CF1092E902AFCF81E08093E902809366
:103C60005F048091E3029091E4029093E2028093DA
:103C7000E102A1CF64E670E080E090E00E942004C1
:103C800080910F01909110010B9731F58091FF0405
:103C9000882309F0F89482E10E9453048C018091FA
:103CA000FF04882309F078940115110509F4ADC0CB
:103CB00080E090ECA9E7B4EC8093F2049093F304D5
:103CC000A093F404B093F5048093F6049093F70462
:103CD000A093F804B093F90480910F019091100122
:103CE000469731F58091FF04882309F0F89481E02C
:103CF0000E9453048C018091FF04882309F078947A
:103D00000115110509F4E2C080E090ECA9E7B4ECDC
:103D10008093F2049093F304A093F404B093F50419
:103D20008093F6049093F704A093F804B093F904F9
:103D300064E670E080E090E00E942004012B09F02E
:103D40003ACF4091F6045091F7046091F8047091D5
:103D5000F90421E0CE0107960E940A0D6DEC71E096
:103D6000CE0101960E943E0CBE01695F7F4FCE01DD
:103D700001960E947F0B68E172E00E94690BBC0112
:103D800088EA94E00E941E0CCE0101960E94ED0A82
:103D90004091F2045091F3046091F4047091F504A1
:103DA00021E0CE0101960E940A0DBE016F5F7F4F98
:103DB000CE0107960E94A20ACE0101960E94ED0A4A
:103DC0006CE172E0CE0101960E943E0CBE01695F7B
:103DD0007F4FCE0101960E947F0B6FE172E00E943F
:103DE000690BBC0188EA94E00E94920BCE01019617
:103DF0000E94ED0A64E670E080E090E00E942004FA
:103E0000CE0107960E94ED0AD6CE1091FA04E090FA
:103E1000FB046E2D70E090E080E00E945B2D2DECA5
:103E20003CEC4CEC5DE30E94BA2D4B015C01612F30
:103E300070E090E080E00E945B2D9B01AC01C50129
:103E4000B4010E942C2F6093F2047093F3048093CA
:103E5000F4049093F5040091FC04F090FD04602FAD
:103E60006F7770E090E080E00E945B2D4B015C0179
:103E70006F2D70E090E080E00E945B2D2DEC3CEC1B
:103E80004CEC5DE30E94BA2D9B01AC01C501B4016D
:103E90000E942C2F07FD18C06093F6047093F7045E
:103EA0008093F8049093F9041E0D100F1F0D81E00C
:103EB00090E02091FE04121302C090E080E0002701
:103EC0001127081B190B08CF9058E6CF1091FB045F
:103ED0000091FA046091FA047091FB047627672739
:103EE000762790E080E00E94592D2DEC3CEC4CECC4
:103EF0005DE30E94BA2D6093F2047093F304809303
:103F0000F4049093F504E090FD04F090FC046F2D10
:103F10006F77762F6E2D90E080E00E94592D2DEC6A
:103F20003CEC4CEC5DE30E94BA2DF7FC18C06093AA
:103F3000F6047093F7048093F8049093F904100F3B
:103F40001E0D1F0D81E090E02091FE04121302C0AF
:103F500090E080E000271127081B190BE9CE90584C
:103F6000E6CF80910E01882309F425CE0E947D08BA
:103F70006B017C010E9465089C0150E040E080914B
:103F8000DC049091DD04281B390B41095109A091F3
:103F9000DA04B091DB040E94B02E4B015C019FE07B
:103FA000B594A794979487949A95D1F76091D40487
:103FB0007091D504072E000C880B990B2BE0660F2F
:103FC000771F881F991F2A95D1F72091D604309129
:103FD000D704032E000C440B550B280D391D4A1D28
:103FE0005B1D0E94912ECA01B901680D791D8A1DC1
:103FF0009B1D685F7F4F8F4F9F4F34E0959587954E
:10400000779567953A95D1F70E945B2D2B013C017E
:104010006091150470911604809117049091180412
:104020000E945B2D4B015C010E947D080E945B2D6C
:10403000A50194010E940A3021E03EED42E45EE3D6
:104040000E94E6304B015C01C701B6010E945B2D66
:1040500020E030E048EC52E40E940A30AB01BC01A1
:1040600022E0CE0101960E940A0DBE016F5F7F4FD4
:104070008AE894E00E94A20ACE0101960E94ED0A0D
:1040800043E050E063EB71E08AE894E00E941F0B8C
:104090006AE874E080E994E00E941E0C62E971E035
:1040A000CE0101960E943E0C6AE874E0CE010196B2
:1040B0000E947F0BBC018AE894E00E941E0CCE0196
:1040C00001960E94ED0A6DE472E088EA94E00E9495
:1040D000990B20E030E040E251E4C301B2010E94BC
:1040E0000A30AB01BC0121E0CE0101960E940A0D0D
:1040F000BE016F5F7F4F88EA94E00E94920BCE0171
:1041000001960E94ED0A45E050E061E272E088EA23
:1041100094E00E941F0BA501940160E070E080E82C
:104120009FE30E942B2F20E03AE24DE257E40E94E9
:10413000BA2DAB01BC0121E0CE0107960E940A0D09
:10414000BE01695F7F4FCE0101960E94350C67E288
:1041500072E0CE0101960E94690BBC0188EA94E0EE
:104160000E94920BCE0101960E94ED0ACE010796A5
:104170000E94ED0A6AE874E0CE0101960E94350CB7
:104180006AE671E0CE0101960E94690B68EA74E06C
:104190000E947F0BBC0188EA94E00E941E0CCE01B5
:1041A00001960E94ED0A65E070E080E090E04ECD5F
:1041B00081E0809317010E94D6048C0160E572E0D3
:1041C00088EA94E00E94990B60E074E0601B710B38
:1041D000CE0101960E94F20BBE016F5F7F4F88EA0D
:1041E00094E00E94920BCE0101960CCE60E672E044
:1041F00088EA94E00E94990B0E94D604BC01E8CFA3
:1042000080910E01882309F4D6CC8091E90288239D
:1042100029F082E090E00E94980ECDCC20E030E0C2
:104220004AE754E46091000170910101809102011C
:10423000909103010E94BA2D0E947C304B015C01D9
:1042400020E030E04AE754E46091130170911401DA
:1042500080911501909116010E94BA2D0E947C3028
:104260006B017C0139EEC31633E0D306E104F1049F
:104270002CF084E1C82ED12CE12CF12C0E944505B4
:1042800060935C0270935D0280935E0290935F0284
:104290000E9445052B013C0180915C0290915D02DA
:1042A000A0915E02B0915F02A3019201281B390B1D
:1042B0004A0B5B0BDA01C90188159905AA05BB05F4
:1042C0000CF079CC83E090E00E94980E0E944505A6
:1042D000DC01CB0184199509A609B7098C159D0548
:1042E000AE05BF05ACF6A7019601281B390B4A0B9A
:1042F0005B0BCA01B9010E942004CACF80910E0154
:10430000882309F458CC8091E902882359F021E0F0
:1043100030E040E050E06AE070E080E090E00E9431
:10432000891949CC20E030E04AE754E4609100016B
:104330007091010180910201909103010E94BA2DB8
:104340000E947C306B017C0120E030E04AE754E4BD
:1043500060911301709114018091150190911601E3
:104360000E94BA2D0E947C30A7019601D8CFF0E0C0
:10437000E0E0099520CC8091590418160CF055C046
:1043800081E08093570469E772E088EA94E00E9434
:10439000990B80915704882309F44AC069E272E0BE
:1043A000CE0101960E943E0C68EA74E0CE010196AF
:1043B0000E947F0BBC0188EA94E00E941E0CCE0193
:1043C00001960E94ED0A68EA74E0CE0101960E940F
:1043D000350CCE0101960E94A70CCE0101960E94D9
:1043E000ED0A68EE73E080E090E00E942004809186
:1043F000570481110E94352262E571E088EA94E059
:104400000E94E80B8091E90280935F048111D3CB75
:104410006AEB71E08CE994E00E94E80B86EE9FEF76
:104420009093E4028093E302C6CB10925704ABCF83
:1044300061E372E0CE0101960E943E0C68EA74E0EE
:10444000CE0101960E947F0BBC0188EA94E00E9495
:104450001E0CCE0101960E94ED0AD4CF6BE672E0ED
:1044600088EA94E00E94990BA6CB0F931F93CF93F9
:10447000DF9307E514E0D0E0C0E00A5F1F4F8091B2
:104480005904082E000C990BC817D9076CF4F801D1
:10449000878190850E947B1D68EE73E080E090E04C
:1044A0000E9420042196E9CFDF91CF911F910F91B7
:1044B00008951F920F920FB60F9211242F933F93DE
:1044C0004F935F936F937F938F939F93AF93BF931C
:1044D000EF93FF9380E693E00E94C002FF91EF917B
:1044E000BF91AF919F918F917F916F915F914F910C
:1044F0003F912F910F900FBE0F901F9018951F9214
:104500000F920FB60F9211242F938F939F93EF93D7
:10451000FF93E0917003F09171038081E091760345
:10452000F091770382FD1BC09081809179038F5FAA
:104530008F7320917A03821741F0E0917903F0E0C4
:10454000E05AFC4F958F80937903FF91EF919F91F3
:104550008F912F910F900FBE0F901F901895808113
:10456000F4CF1F920F920FB60F9211242F933F9307
:104570008F939F93AF93BF938091D6029091D70270
:10458000A091D802B091D9023091D50223E0230F37
:104590002D3758F50196A11DB11D2093D5028093AA
:1045A000D6029093D702A093D802B093D9028091FB
:1045B000DA029091DB02A091DC02B091DD0201965B
:1045C000A11DB11D8093DA029093DB02A093DC025F
:1045D000B093DD02BF91AF919F918F913F912F9149
:1045E0000F900FBE0F901F90189526E8230F02968C
:1045F000A11DB11DD2CF1F920F920FB60F921124A1
:104600002F933F934F935F936F937F938F939F93DA
:10461000AF93BF93EF93FF938091B900887F80366B
:1046200009F44AC0F0F5883209F4A7C018F58031C2
:1046300009F49BC0B8F4882309F4F9C0883009F460
:1046400094C0FF91EF91BF91AF919F918F917F9116
:104650006F915F914F913F912F910F900FBE0F90EF
:104660001F901895883109F488C0803251F78093E3
:10467000340314C0803409F49DC040F48033B9F38E
:104680008833F9F68093340385ECB0C0803509F4A3
:1046900085C0883509F496C0883499F60E94600E6A
:1046A000D0CF883909F48CC038F5883729F050F418
:1046B000883611F0803729F683E080933603109214
:1046C000D40257C0883809F47BC0803919F080388B
:1046D00009F0B7CF8091D402803208F071C0E09128
:1046E000D40281E08E0F8093D4028091BB00F0E071
:1046F000EC54FD4F80833DC0803B39F0E0F4803ABC
:1047000009F479C0883A09F09CCF84E0809336039D
:104710001092B3021092B202E091EC02F091ED021D
:1047200009958091B20281110FC081E08093B2029D
:104730001092920209C0803C09F4A6CF883C09F48B
:10474000A3CF883B09F07DCFE091B30281E08E0FCB
:104750008093B302F0E0EE56FD4F80818093BB0062
:104760009091B3028091B20229C08091110380938D
:10477000BB0085EC8093BC0064CF909133038091A3
:104780003203981758F5E091330381E08E0F809340
:104790003303F0E0EE5EFC4F8081E9CFE09133031C
:1047A00081E08E0F809333038091BB00F0E0EE5EDA
:1047B000FC4F808390913303809132039817C8F2A5
:1047C00085E8D8CFE091330381E08E0F80933303E7
:1047D0008091BB00F0E0EE5EFC4F8083809135035A
:1047E00081115CCF81E08093100384EA8093BC0048
:1047F0001092360326CF85EC8093BC0010923603CE
:104800008091D402803230F4E091D402F0E0EC5494
:10481000FD4F10826091D40270E0E091EA02F091C5
:10482000EB0284EB92E009951092D4020ACF109229
:10483000340334CFCF93DF93E0E6F3E013821282A8
:1048400088EE93E0A0E0B0E084839583A683B783ED
:1048500022E231E03183208325EC30E03587248764
:1048600024EC30E03787268720EC30E0318B208B3A
:1048700021EC30E0338B228B22EC30E0358B248B23
:1048800026EC30E0378B268B118E128E138E148E11
:10489000EDEFF3E01382128284839583A683B783BE
:1048A00084E391E0918380831092FF04EEEDF4E0C5
:1048B000C1E0C083118283EC9BEAA6E7BBE382835D
:1048C0009383A483B58388ED9BE6A6E7BBE3868349
:1048D0009783A087B18782EF94EEA4E6BBE382873B
:1048E0009387A487B587EEEAF4E086E491E09183AC
:1048F00080838FEF9FEFDC01858B968BA78BB08F2A
:1049000062E571E088EA94E00E943E0C62E571E0A5
:1049100082EA94E00E943E0C62E571E08CE994E04A
:104920000E943E0C62E571E086E994E00E943E0C34
:1049300062E571E080E994E00E943E0C62E571E07E
:104940008AE894E00E943E0C6AE372E084E894E016
:104950000E943E0C61E472E08EE794E00E943E0CFF
:10496000E7E5F4E0108285E08183128214821382ED
:104970001682158217821086E9E0F4E086E190E065
:10498000918380838CE79CE8A1E0B0E084879587E1
:10499000A687B78781EA97E6A3E3BDEB808B918B6F
:1049A000A28BB38B86E696E6A6EABFE3848B958B53
:1049B000A68BB78BC0A389E190E092A381A3C3A388
:1049C00080E090E4ACE1B5E484A395A3A6A3B7A3EB
:1049D00010A611A612A613A6A5E3B4E080E1ED018E
:1049E00019928A95E9F714AE15AE16AE17AE10926D
:1049F000490410924A0410924B0410924C041092F5
:104A00004D0410924E0410924F04109250041092D4
:104A1000510410925204109253041092540481E0F5
:104A200090E09093560480935504DF91CF910895C0
:104A3000CF93DF93CDB7DEB7AE970FB6F894DEBF56
:104A40000FBECDBF789484B5826084BD84B581608B
:104A500084BD85B5826085BD85B5816085BD809149
:104A60006E00816080936E001092810080918100C1
:104A700082608093810080918100816080938100B9
:104A8000809180008160809380008091B10084607B
:104A90008093B1008091B00081608093B0008091DC
:104AA0007A00846080937A0080917A00826080939B
:104AB0007A0080917A00816080937A0080917A00F8
:104AC000806880937A001092C10061E08EE00E94BD
:104AD000CA03E0917003F091710382E08083E0915A
:104AE0006C03F0916D031082E0916E03F0916F03FF
:104AF0008FEC808310927803E0917403F09175033A
:104B000086E08083E0917203F0917303808180617D
:104B10008083E0917203F0917303808188608083C9
:104B2000E0917203F0917303808180688083E0914B
:104B30007203F091730380818F7D808361E080E157
:104B40000E94CA0360E080E10E949C0361E08EE065
:104B50000E949C0368EC70E080E090E00E942004DA
:104B600084E690E090931201809311010E947B2EC5
:104B70008093DE0285E690E00E947B2E8093DF0228
:104B80000091DE021091DF02B801012E000C880BAB
:104B9000990B0E945B2D9B01AC010E948031811119
:104BA00006C00B5011090C30110508F4B8C084E69A
:104BB00090E00E94BD1137E5E32E34E0F32E67014B
:104BC0000EE110E0C8010E947B2EF60181936F0177
:104BD0000F5F1F4F07321105A9F710915804612F7D
:104BE000012E000C770B880B990B0E945B2D9B010B
:104BF000AC010E948031811103C0153009F4BAC0A4
:104C00008EE190E00E94E61168EC70E080E090E0B8
:104C10000E94200467E273E088EA94E00E94990B06
:104C200068EA74E0CE0101960E94350CCE0101962F
:104C30000E94A70CCE0101960E94ED0A0E949F05DA
:104C400064E670E080E090E00E94200483E08093BE
:104C5000C7040E949F0580ED0E942308853509F452
:104C600097C06BE173E088EA94E00E94990B109280
:104C70000E0168EA74E0CE0101960E94350CCE0167
:104C800001960E94A70CCE0101960E94ED0AF12C1C
:104C9000E12C9AE2C92ED12C28EE422E23E0522E8E
:104CA000612C712C01E080E0A82E80E0B82E62E536
:104CB00071E0CE0189960E943E0C10E080E693E000
:104CC0000E94A002181619060CF00CC111110AC19D
:104CD00080E693E00E947E028A3009F0B3C1109111
:104CE000E002112309F4C3C180919A0490919B04BE
:104CF000892B09F4B5C16AE472E0CE0101960E94E5
:104D00003E0CBE01675D7F4FCE0101960E947F0B76
:104D10000E945D02CE0101960E94ED0AA1C149E008
:104D2000E42E44E0F42E04E610E0C8010E947B2E3D
:104D3000F70181937F010F5F1F4F023B1105A9F718
:104D40008091090490910A049093100180930F01BF
:104D50006BE074E0CE0101960E943E0CBE016F5FD5
:104D60007F4F84E894E00E94A20ACE0101960E943F
:104D7000ED0A21CF0EE110E0C8010E947B2EF70161
:104D800081937F010F5F1F4F05341105A9F73CCFB9
:104D90008AEA0E9440089093C9048093C8048CEA70
:104DA0000E9440089093CB048093CA048EEA0E942C
:104DB00040089093CD048093CC0480EB0E9440087F
:104DC0009093D9048093D80482EB0E94400890937A
:104DD000DB048093DA0484EB0E9440089093DD04A6
:104DE0008093DC0486EB0E9440089093CF0480936C
:104DF000CE0488EB0E9440089093D1048093D004A5
:104E00008AEB0E9440089093D3048093D2048CEBE9
:104E10000E9440089093D5048093D4048EEB0E94A6
:104E200040089093D7048093D60464EF71E080E04B
:104E300090E00E9420040E949F0580E00E94F907F4
:104E400080E10E94F90788E00E94F9070E949F050F
:104E50008EE10E941A0262E08DEF93E00E94CA0781
:104E600060E08DEF93E00E94CA070E94D7058EE1B3
:104E70000E941A0261E08DEF93E00E94CA0760E28F
:104E80008DEF93E00E94CA070E94D70580E290E070
:104E90009093B2048093B10480E090E8A9E8B4E470
:104EA00080930A0190930B01A0930C01B0930D0124
:104EB00080E090E0A5E7B4E48093060190930701B9
:104EC000A0930801B0930901BE016F5F7F4F8EEA86
:104ED00094E00E94400D64EF71E080E090E00E9459
:104EE0002004D5CE8DA59EA5892B51F080E693E0B8
:104EF0000E942F0364E170E080E090E00E942004B3
:104F0000BE01675D7F4F86E994E00E94A20ACE0150
:104F100089960E94ED0A62E571E088EA94E00E94B9
:104F2000E80B80919A0490919B048130910509F0DF
:104F3000C6C066E974E082EA94E00E941E0C0E94FA
:104F4000650A62EA74E0CE0101960E94350C8D81FB
:104F50009E81892B09F4A5C0E981FA81309709F473
:104F6000A0C08081823409F484C0833409F48EC0E7
:104F7000813409F096C063E572E086E994E00E940E
:104F8000E80BCE0101960E94ED0A86E994E00E94AA
:104F90007C0ACB010E947B1D8091E902882309F4E1
:104FA0003FC00E944505A30192010E94FA2ECA014A
:104FB000B9010E94592D2091E5023091E6024091FD
:104FC000E7025091E8020E942B2F209113013091AB
:104FD000140140911501509116010E94D930181604
:104FE000FCF48091E3029091E4024A9609F4B8C07F
:104FF0008091E1029091E2020E947B1D0E94450592
:10500000A30192010E94FA2ECA01B9010E94592DF2
:105010006093E5027093E6028093E7029093E802C2
:105020006AE070E080E090E00E942004A114B104E6
:1050300009F43DCE0E94AC02882309F438CE0E94C8
:10504000000031CE8D3009F44ACE89831A8241E0C6
:1050500050E0BE016F5F7F4FCE0189960E941F0B0B
:105060006AE070E080E090E00E94200427CE11E02A
:10507000F7CF66E572E086E994E00E94E80B1092B3
:10508000E9028CEF9FEF0E947B1D7BCF69E572E008
:1050900086E994E00E94E80B0093E9028DEF9FEF10
:1050A000F2CFBE016F5F7F4F86E994E00E941E0C35
:1050B0006AE070E080E090E00E94200462CF0497F4
:1050C00068F56BEB71E0CE0101960E943E0CBE01CB
:1050D0006F5F7F4F86E994E00E94870A182FCE0108
:1050E00001960E94ED0A1123C9F080919A049091D3
:1050F0009B04029788F0E0919604F0919704309712
:1051000059F0818180330CF4845E9601281B3109AB
:1051100087FD3395C9013ECF80E0F6CF66E974E0A4
:1051200082EA94E00E941E0C0E94650A63E473E028
:10513000CE0101960E94BE0BBE016F5F7F4F82EAD7
:1051400094E00E94870A182FCE0101960E94ED0A72
:10515000112319F0F70109951FCF0E940F121CCFE0
:1051600080915704882309F449CF0E94352246CF05
:105170008EE794E00E94ED0A84E894E00E94ED0A34
:105180008AE894E00E94ED0A80E994E00E94ED0A2A
:1051900086E994E00E94ED0A8CE994E00E94ED0A11
:1051A00082EA94E00E94ED0A88EA94E00C94ED0A09
:1051B000EF920F931F93CF93DF93E80134E047FD05
:1051C00034E1042E000C550B57FF03C05195419557
:1051D0005109E32E022F242FAE010E949C29CE01FB
:1051E000DF91CF911F910F91EF9008956627772758
:1051F0000C94FB2A1F93FC0199278827BC01E89493
:1052000011911032E9F3193010F01E30C8F31B323F
:1052100051F01D3249F4689406C00E944B29610F79
:10522000711D811D911D119110531A30B0F33EF480
:1052300090958095709561957F4F8F4F9F4F1F91EF
:105240000895FB01DC0105900D920020E1F708951F
:10525000FC0105900020E9F7809590958E0F9F1F27
:105260000895BB274A3031F4992322F4BDE290958A
:1052700081959F4F0C948329BB272A3051F49923A1
:1052800042F4BDE290958095709561957F4F8F4F68
:105290009F4F0C946129592F482F372F262F660FC7
:1052A000771F881F991F660F771F881F991F620F2E
:1052B000731F841F951F660F771F881F991F0895FE
:1052C000BB27FA01A62F6217710581059105330BE3
:1052D00030FB66F0AA27660F771F881F991FAA1F49
:1052E000A21710F0A21B63953850A9F7A05DAA334E
:1052F00008F0A95DA19336F7B111B1931082CA01EC
:105300000C94442DBB27FB015527AA27880F991F12
:10531000AA1FA41710F0A41B83955051B9F7A05DE4
:10532000AA3308F0A95DA193009779F7B111B19361
:105330001192CB010C94442DA9E0B0E0E2EAF9E22D
:105340000C94C92E6A01F22EB02E102FFBE3AF2E63
:10535000A01608F41BE31F5F012F27E0AE014F5F8B
:105360005F4F0E944B2CBC018981982F997091301E
:1053700009F43FC09BE2E1FC04C09E2D9170E0FC6B
:105380003AC05E2D5071E82FE87083FF46C084E07C
:10539000911101C083E0EF2DE81B8F1508F0E0E0CC
:1053A000D6018E2F20E2552351F1992329F0D60101
:1053B0009C93C60101966C0196012D5F3F4FE2FE62
:1053C00024C08EE4D6018C9391E411969C9311979E
:1053D00012968C93D9018E2F90E281111BC0E20F9F
:1053E000F32FF11D10828EEF9FEF2996ECE00C94C5
:1053F000E52E9DE2C6CF90E2C4CF2D93815081115E
:10540000FCCFCE0ED11CE0E0D0CF8EE6D6018C933F
:1054100091E6DBCF9D938150E0CF482F447082FF0F
:105420003DC084E0911101C083E08F1510F4EF2D91
:10543000E81BD6018E2F20E2552309F1992329F08C
:10544000D6019C93C60101966C0196012D5F3F4FDA
:10545000E2FE1BC089E4D6018C938EE411968C93F6
:10546000119786E412968C93D9018E2F90E28823AF
:1054700009F4B5CF9D938150FACF2D9381508111BE
:10548000FCCFCE0ED11CE0E0D9CF89E6D6018C93BB
:105490008EE611968C93119786E6E4CF9B0177FFF9
:1054A00002C030E020E0A1E0B0E0911102C0B0E025
:1054B000A0E0F9013196AE0FBF1F8B2C912CBB20C1
:1054C00009F461C05401EFEFAE1ABE0AAA0DBB1D6C
:1054D000FA161B0619F014F04F2D4A1B511188C003
:1054E000E3FC59C07601A42FB0E2A1114FC0C40E55
:1054F000D11C992309F45BC040E0D6011196F60156
:1055000090836D01552309F448C0012F060F9A813D
:10551000582F507184FF03C0913309F401501016C5
:105520000CF047C0093008F008E0EEE2FE2E5B0107
:10553000A01AB10885019194819491082F3F3207F8
:1055400029F4D601FC92F60131966F0162177307B8
:1055500094F1021713077CF5DB01A21BB30BAA24FD
:10556000A394B12CAC0EBD1EAA0DBB1D11968C913F
:1055700021503109D601119628153905F4F0F601AC
:1055800080836D01DBCFB12CA12CA0CFF701B193AB
:105590007F01A150AACF9111B0CFD601942F50E333
:1055A00002C05D9391509111FCCFC40ED11C40E01C
:1055B000ACCF01E0BACF80E3DBCF6217730731F4E1
:1055C000963388F4953311F4552369F0F6018083FE
:1055D000FD01842F90E2811108C0A40FB11D1C921F
:1055E00090E080E002CF81E3F1CF91938150F3CF3F
:1055F000911183CF8ACFB0E0A0E0E1E0FBE20C9410
:10560000C92E5C017B016115710519F0DB018D93D9
:105610009C9385010F5F1F4FF501D0818D2F90E086
:105620000E94232D6C01892BB9F5DD32B9F50F5F8E
:105630001F4FD5011196DC91C1E05801F1E0AF1A7E
:10564000B10843E050E060E271E0C5010E942C2DFA
:10565000892B69F5680182E0C80ED11C45E050E055
:105660006BE171E0C6010E942C2D892B21F46801A9
:1056700097E0C90ED11CE114F10419F0D701CD92C5
:10568000DC9260E070E080E89FEFC111FFC060E055
:1056900070E080E89FE7FAC05801BBCFDB3229F405
:1056A00085010E5F1F4FF501D181C0E0C6CF43E0F9
:1056B00050E068E171E0C5010E942C2D892BE9F0D2
:1056C000F80110E000E020E030E0A9015F01B0ED5A
:1056D0008B2E8D0E89E08815C8F19C2E689491F868
:1056E0008C2F8870C2FF16C0811102C00F5F1F4F40
:1056F0003196D501DC91C92DE9CFE114F10429F0EF
:105700000E5F1F4FF7011183008360E070E080ECB3
:105710009FE7BCC0882311F001501109A5E0B0E05B
:105720000E94B02E9B01AC01220F331F441F551F56
:10573000280D311D411D511D283999E939074907A7
:1057400099E15907A8F2C6609C2ED2CFAEEF8A121B
:1057500006C0C3FD3CC09C2E689493F8C9CFDF7D82
:10576000D534A9F580818D3239F4C061DF011296FC
:10577000818162E070E006C0DF018B32C1F31196D7
:1057800061E070E080535D01A61AB70A8A30F8F430
:10579000E0E8CE16ECE0DE065CF4B601660F771F9B
:1057A000660F771FC60ED71ECC0CDD1CC80ED11C91
:1057B0005D01FFEFAF1ABF0A8C9180538A30A8F1C8
:1057C000C4FF03C0D194C194D1080C0D1D1DC1FFAD
:1057D00009C0E114F10431F081E0A81AB108D70141
:1057E000AD92BC92CA01B9010E94592DC370C33059
:1057F00009F490584B015C0120E030E0A9010E94BF
:10580000542D882309F440C0CFE4D1E017FF05C030
:10581000119501951109C7E3D1E06E01B8E1CB1AEA
:10582000D10880E2E82EF12C0FC0D501B1CFFE01E6
:1058300025913591459154910E191F09C501B40167
:105840000E94BA2D4B015C01D501C4010E151F0544
:1058500074F72497F594E794CC16DD06A9F78A2F00
:10586000880F8B2F881F8F3F49F020E030E0A9017F
:10587000C501B4010E94542D811106C082E290E05E
:105880009093010580930005C501B401CDB7DEB743
:10589000ECE00C94E52E283008F027E03327DA01FD
:1058A000990F311D87FD916000966105710539F4EE
:1058B00032602E5F3D9330E32A95E1F708959F3FD4
:1058C00030F080387105610509F03C5F3C5F3D9325
:1058D000913008F08068911DDF93CF931F930F9351
:1058E000FF92EF92192F987F9695E92F96959695AE
:1058F000E90FFF27E355FE4F99273327EE24FF24B6
:10590000A701E70105900894079428F4360FE71ED5
:10591000F81E491F511D660F771F881F991F069497
:10592000A1F70590079428F4E70EF81E491F561FAB
:10593000C11D770F881F991F661F0694A1F7059058
:10594000079428F4F80E491F561FC71FD11D880F52
:10595000991F661F771F0694A1F70590079420F4FE
:10596000490F561FC71FD81F990F661F771F881F23
:105970000694A9F784911095177041F0D695C795B4
:1059800057954795F794E7941A95C1F7E3E5F1E049
:1059900068941590159135916591959105907FE2E8
:1059A0007395E118F10A430B560BC90BD009C0F7E8
:1059B000E10CF11E431F561FC91FD01D7EF470332A
:1059C00011F48A95E6CFE894015030F0080F0AF4FC
:1059D0000027021708F4202F2395022F7A3328F08E
:1059E00079E37D932A95E9F710C07D932A9589F68E
:1059F000069497956795379517951794E118F10ACE
:105A0000430B560BC90BD00998F023957E917395E3
:105A10007A3308F070E37C932013B8F77E917061BD
:105A20007D9330F0839571E37D9370E32A95E1F7E0
:105A30001124EF90FF900F911F91CF91DF91992743
:105A400087FD9095089591110C94272E803219F0BE
:105A500089508550C8F70895FB01DC014150504042
:105A600088F08D9181341CF08B350CF4805E65914B
:105A700061341CF06B350CF4605E861B611171F3B0
:105A8000990B0895881BFCCFDC01FC01672F7191F5
:105A90007723E1F7329704C07C916D937083629114
:105AA000AE17BF07C8F308950E94962D08F481E051
:105AB0000895E89409C097FB3EF490958095709501
:105AC00061957F4F8F4F9F4F9923A9F0F92F96E94A
:105AD000BB279395F695879577956795B795F111BF
:105AE000F8CFFAF4BB0F11F460FF1BC06F5F7F4F5C
:105AF0008F4F9F4F16C0882311F096E911C077236E
:105B000021F09EE8872F762F05C0662371F096E876
:105B1000862F70E060E02AF09A95660F771F881F45
:105B2000DAF7880F9695879597F90895990F0008E9
:105B3000550FAA0BE0E8FEEF16161706E807F9075F
:105B4000C0F012161306E407F50798F0621B730BFA
:105B5000840B950B39F40A2661F0232B242B252B7B
:105B600021F408950A2609F4A140A6958FEF811D1E
:105B7000811D08950E94CD2D0C94412E0E94332E3C
:105B800038F00E943A2E20F0952311F00C942A2E22
:105B90000C94302E11240C94752E0E94522E70F30A
:105BA000959FC1F3950F50E0551F629FF001729FC2
:105BB000BB27F00DB11D639FAA27F00DB11DAA1FD1
:105BC000649F6627B00DA11D661F829F2227B00D1E
:105BD000A11D621F739FB00DA11D621F839FA00DA9
:105BE000611D221F749F3327A00D611D231F849FF9
:105BF000600D211D822F762F6A2F11249F57504050
:105C00009AF0F1F088234AF0EE0FFF1FBB1F661FCA
:105C1000771F881F91505040A9F79E3F510580F093
:105C20000C942A2E0C94752E5F3FE4F3983ED4F327
:105C3000869577956795B795F795E7959F5FC1F737
:105C4000FE2B880F911D9695879597F908959927B2
:105C50008827089597F99F6780E870E060E00895CD
:105C60009FEF80EC089500240A9416161706180674
:105C70000906089500240A94121613061406050650
:105C80000895092E0394000C11F4882352F0BB0FE1
:105C900040F4BF2B11F460FF04C06F5F7F4F8F4F44
:105CA0009F4F089557FD9058440F551F59F05F3F7F
:105CB00071F04795880F97FB991F61F09F3F79F02E
:105CC00087950895121613061406551FF2CF4695B0
:105CD000F1DF08C0161617061806991FF1CF869532
:105CE0007105610508940895E894BB276627772716
:105CF000CB0197F90895F999FECF92BD81BDF89A2D
:105D0000992780B50895262FF999FECF1FBA92BD25
:105D100081BD20BD0FB6F894FA9AF99A0FBE01968C
:105D20000895052E97FB1EF400940E94A82E57FD9F
:105D300007D00E94FA2E07FC03D04EF40C94A82E34
:105D400050954095309521953F4F4F4F5F4F0895A7
:105D500090958095709561957F4F8F4F9F4F0895D7
:105D60000E941C2FA59F900DB49F900DA49F800DA5
:105D7000911D11240895B7FF0C94B02E0E94B02EEF
:105D8000821B930B08952F923F924F925F926F92D6
:105D90007F928F929F92AF92BF92CF92DF92EF92BB
:105DA000FF920F931F93CF93DF93CDB7DEB7CA1B3C
:105DB000DB0B0FB6F894DEBF0FBECDBF09942A8867
:105DC000398848885F846E847D848C849B84AA840F
:105DD000B984C884DF80EE80FD800C811B81AA819C
:105DE000B981CE0FD11D0FB6F894DEBF0FBECDBF67
:105DF000ED010895A1E21A2EAA1BBB1BFD010DC0E7
:105E0000AA1FBB1FEE1FFF1FA217B307E407F5076A
:105E100020F0A21BB30BE40BF50B661F771F881F46
:105E2000991F1A9469F760957095809590959B01DC
:105E3000AC01BD01CF010895A29FB001B39FC00185
:105E4000A39F700D811D1124911DB29F700D811DA6
:105E50001124911D08955058BB27AA270E94432F53
:105E60000C94412E0E94332E38F00E943A2E20F0DE
:105E700039F49F3F19F426F40C94302E0EF4E0957B
:105E8000E7FB0C942A2EE92F0E94522E58F3BA17E2
:105E9000620773078407950720F079F4A6F50C9440
:105EA000742E0EF4E0950B2EBA2FA02D0B01B90124
:105EB00090010C01CA01A0011124FF27591B99F080
:105EC000593F50F4503E68F11A16F040A22F232F8C
:105ED000342F4427585FF3CF469537952795A795DC
:105EE000F0405395C9F77EF41F16BA0B620B730B83
:105EF000840BBAF09150A1F0FF0FBB1F661F771FF4
:105F0000881FC2F70EC0BA0F621F731F841F48F4A8
:105F1000879577956795B795F7959E3F08F0B0CF31
:105F20009395880F08F09927EE0F97958795089518
:105F30000E94332E60F080E891E009F49EEF0E9409
:105F40003A2E28F040E851E071F45EEF0CC00C945A
:105F5000302E0C94742EE92FE0780E94522E40F3DC
:105F6000092E052AB1F3261737074807590738F0D5
:105F70000E2E07F8E02569F0E025E0640AC0EF6323
:105F800007F8009407FADB01B9019D01DC01CA01A1
:105F9000AD01EF930E9421300E94412E0E94DB2F21
:105FA0005F91552339F02BED3FE049E450FD49EC7A
:105FB0000C942C2F0895DF93DD27B92FBF7740E88D
:105FC0005FE31616170648075B0718F4D92F0E94DF
:105FD000DE309F938F937F936F930E947C31E8E62E
:105FE000F0E00E94B2300E94412E2F913F914F91DC
:105FF0005F910E94CD2DDD2351F09058A2EA2AED49
:106000003FE049EC5FE3D0785D270E94432FDF91AA
:106010000C94412E0E941E300C94412E0E943A2E68
:1060200058F00E94332E40F029F45F3F29F00C9481
:106030002A2E51110C94752E0C94302E0E94522E43
:1060400068F39923B1F3552391F3951B550BBB27A7
:10605000AA2762177307840738F09F5F5F4F220FEC
:10606000331F441FAA1FA9F335D00E2E3AF0E0E8E3
:1060700032D091505040E695001CCAF72BD0FE2F2D
:1060800029D0660F771F881FBB1F261737074807C1
:10609000AB07B0E809F0BB0B802DBF01FF27935879
:1060A0005F4F3AF09E3F510578F00C942A2E0C94E5
:1060B000752E5F3FE4F3983ED4F386957795679508
:1060C000B795F7959F5FC9F7880F911D96958795AE
:1060D00097F90895E1E0660F771F881FBB1F6217CD
:1060E00073078407BA0720F0621B730B840BBA0B8B
:1060F000EE1F88F7E09508950E9483306894B111EF
:106100000C94752E08950E945A2E88F09F5798F08F
:10611000B92F9927B751B0F0E1F0660F771F881FAC
:10612000991F1AF0BA95C9F714C0B13091F00E94C6
:10613000742EB1E008950C94742E672F782F882761
:10614000B85F39F0B93FCCF3869577956795B395ED
:10615000D9F73EF490958095709561957F4F8F4F5C
:106160009F4F0895DF93CF931F930F93FF92EF926A
:10617000DF927B018C01689406C0DA2EEF010E9449
:10618000CD2DFE01E894A59125913591459155912C
:10619000A6F3EF010E94432FFE019701A801DA94B4
:1061A00069F7DF90EF90FF900F911F91CF91DF91F2
:1061B00008950E94962D08F48FEF08959B01AC017D
:1061C00060E070E080E89FE30C940A30FA01EE0F83
:1061D000FF1F309621053105A1F16115710561F4AC
:1061E0008038BFE39B0749F168949038810561F0DE
:1061F0008038BFEF9B0741F099234AF5FF3FE10547
:106200003105210519F1E8940894E795D901AA23ED
:1062100029F4AB2FBE2FF85FD0F310C0FF5F70F4EE
:10622000A695E0F7F73950F019F0FF3A38F49F7768
:106230009F930DD00F9007FC9058089546F00C9452
:10624000302E60E070E080E89FE308954FE79F778D
:106250005F934F933F932F930E9416322F913F915C
:106260004F915F910E94BA2D0C948D3119F416F460
:106270000C94302E0C94BF310E945A2EB8F39923FF
:10628000C9F3B6F39F57550B87FF0E94CD31002409
:10629000A0E640EA900180585695979528F4805CD6
:1062A000660F771F881F20F026173707480730F43E
:1062B000621B730B840B202931294A2BA695179456
:1062C0000794202531254A2758F7660F771F881F26
:1062D00020F026173707480730F4620B730B840B46
:1062E000200D311D411DA09581F7B901842F9158D2
:1062F000880F9695879508959B01AC010C94BA2D53
:106300000E94962D880B990B089529F416F00C9491
:106310002A2E0C94742E0C94302E0E945A2EA8F320
:106320009638A0F707F80F92E8942BE33AEA48EB87
:106330005FE70E94D02D0F920F920F924DB75EB77C
:106340000F920E945E32E5E9F0E00E94B2304F9178
:106350005F91EF91FF91E595EE1FFF1F49F0FE570A
:10636000E0684427EE0F441FFA95E1F74195550B7D
:106370000E94D8310F9007FE0C94DE3008959F3FA5
:1063800031F0915020F4879577956795B795880FF0
:10639000911D9695879597F9089591505040660FF5
:1063A000771F881FD2F708950C942A2E0C94BF31C2
:1063B0000E945A2ED8F39923C9F3940F511DA3F3C9
:1063C0009150504094F059F0882332F0660F771FB7
:1063D000881F91505040C1F79E3F51052CF7880F00
:1063E000911D9695879597F908955F3FACF0983E7B
:1063F0009CF0BB27869577956795B79508F4B160B3
:106400009395C1F7BB0F58F711F460FFE8CF6F5FAA
:106410007F4F8F4F9F4FE3CF0C94752E16F00C9447
:10642000BF310C94302E68940C942A2E0E945A2E60
:10643000A8F39923C1F3AEF3DF93CF931F930F9388
:10644000FF92C92FDD2788232AF02197660F771F37
:10645000881FDAF720E030E040E85FEB9FE38839FF
:1064600020F0803E38F021968F770E942C2FEDEBA4
:10647000F0E004C00E942C2FEAEEF0E00E94B2305F
:106480008B01BE01EC01FB2E6F5771097595771FCB
:10649000880B990B0E945B2D28E132E741E35FE313
:1064A0000E94CD2DAF2D9801AE01FF900F911F914D
:1064B000CF91DF910E94432F0C94412EFA01DC0111
:1064C000AA0FBB1F9B01AC01BF5728F4222733271B
:1064D0004427507820C0B75190F4AB2F0024469544
:1064E00037952795011CA395D2F3002071F0220F58
:1064F000331F441FB395DAF30ED00C942B2F613069
:106500007105A0E88A07B94630F49B01AC01662703
:10651000772788279078309621F020833183428333
:1065200053830895DB018F939F930E94B02EBF91F8
:10653000AF91A29F800D911DA39F900DB29F900DD2
:1065400011240895AA1BBB1B51E107C0AA1FBB1F42
:10655000A617B70710F0A61BB70B881F991F5A95EF
:10656000A9F780959095BC01CD010895EE0FFF1F0E
:106570000590F491E02D09940F931F93CF93DF932F
:106580008230910510F482E090E0E0910405F091F2
:10659000050530E020E0B0E0A0E0309799F4211547
:1065A000310509F44AC0281B390B24303105D8F5D0
:1065B0008A819B816115710589F1FB019383828337
:1065C000FE0111C040815181028113814817590792
:1065D000E0F04817590799F4109761F012960C9360
:1065E000129713961C933296CF01DF91CF911F9192
:1065F0000F9108950093040510930505F4CF21151C
:10660000310551F04217530738F0A901DB019A0117
:10661000BD01DF01F801C1CFEF01F9CF909305056E
:1066200080930405CDCFFE01E20FF31F8193919378
:106630002250310939832883D7CF20910205309128
:106640000305232B41F420911A0130911B01309353
:10665000030520930205209118013091190121159D
:10666000310541F42DB73EB740911C0150911D01F9
:10667000241B350BE0910205F0910305E217F307A7
:10668000A0F42E1B3F0B2817390778F0AC014E5FA2
:106690005F4F2417350748F04E0F5F1F50930305D7
:1066A00040930205819391939FCFF0E0E0E09CCF6F
:1066B000CF93DF930097E9F0FC01329713821282A7
:1066C000A0910405B0910505ED0130E020E01097A0
:1066D000A1F420813181820F931F20910205309116
:1066E00003052817390709F061C0F0930305E0930B
:1066F0000205DF91CF910895EA01CE17DF07E8F593
:106700004A815B819E0141155105B1F7E901FB8387
:10671000EA8349915991C40FD51FEC17FD0761F425
:10672000808191810296840F951FE9019983888366
:10673000828193819B838A83F0E0E0E012968D91C1
:106740009C9113970097B9F52D913C911197CD012C
:106750000296820F931F209102053091030528179E
:10676000390739F6309751F5109205051092040556
:10677000B0930305A0930205BCCFD383C2834081AD
:106780005181840F951FC817D90761F44E5F5F4F81
:1067900088819981480F591F518340838A819B8149
:1067A000938382832115310509F0B0CFF09305055D
:1067B000E09304059ECFFD01DC01C0CF138212825D
:1067C000D7CFB0E0A0E0E7EEF3E30C94C52E8C0148
:1067D000009751F4CB010E94BC328C01C801CDB7A7
:1067E000DEB7E0E10C94E12EFC01E60FF71F9C01FF
:1067F00022503109E217F30708F49DC0D901CD9169
:10680000DC911197C617D70798F0C530D10530F342
:10681000CE0104978617970708F3C61BD70B22975C
:10682000C193D1936D937C93CF010E945833D6CFFF
:106830005B01AC1ABD0A4C018C0E9D1EA091040593
:10684000B0910505512C412CF12CE12C109731F51C
:1068500080910205909103058815990509F05CC0A7
:106860004616570608F058C08091180190911901FA
:10687000009741F48DB79EB740911C0150911D01C6
:10688000841B950BE817F90708F055C0F093030532
:10689000E0930205F90171836083A0CF8D919C91F3
:1068A000119712966C90129713967C901397A815D7
:1068B000B90559F56C0142E0C40ED11CCA14DB04C1
:1068C00020F1AC014A195B09DA011296159780F0A4
:1068D0006282738251834083D9016D937C93E1146A
:1068E000F10471F0D7011396FC93EE93129776CFD3
:1068F00022968C0F9D1FF90191838083F301EFCFC6
:10690000F0930505E093040569CF4816590608F48D
:106910002C017D01D3019ACFCB010E94BC327C01B6
:10692000009749F0AE01B8010E94A634C8010E9448
:106930005833870153CF10E000E050CF91110895F4
:1069400081568A5108F4805285580895FB01DC0174
:1069500002C001900D9241505040D8F70895FB01BC
:10696000DC0101900D920020E1F70895FB01DC01AC
:106970004150504030F08D910190801919F4002061
:10698000B9F7881B990B0895FB01DC014150504079
:1069900048F001900D920020C9F701C01D924150AE
:1069A0005040E0F70895FB0151915523A9F0BF0134
:1069B000DC014D9145174111E1F759F4CD010190EA
:1069C000002049F04D9140154111C9F3FB014111DF
:1069D000EFCF81E090E00197089511E0C9ECD1E09C
:1069E00004C0FE010E94B6322196CA3CD107C9F705
:1069F000F894FFCF0000A040C8000000754400805C
:106A0000894401160064000000F041010000060501
:106A1000800000000000E20227026F022F03A002A4
:106A20007E02920200000000CA079D070B088D0736
:106A30005205F4018E07000000005105F50A5905C2
:106A40008D0D400D0D0A00484D4335383833004355
:106A50006F6D706173733A200028646567292000A8
:106A60004E200045005320005700732000296D4739
:106A700000203D3E0056657273696F6E3A20002318
:106A8000007300534C20503D005061206973207505
:106A90006E6C696B656C792100536561206C65765D
:106AA000656C20503D0020685061004950414444CD
:106AB0000023495020616464726573733A20004E6C
:106AC00045543D0055565A002C0023496E636F72A1
:106AD0007265637421204D533D3132334433443564
:106AE00000496E636C2E20616E672E287820792015
:106AF0007A292F6465673A20003E6128782C792C2A
:106B00007A292F673A00613D002067006F4320001B
:106B1000483D0025006F4320413D006D0023456E38
:106B200061626C65002344697361626C6500414E6B
:106B30004D4C3033004E616E6F41326734007365E7
:106B40007269616C3A20002D35002D34002D330020
:107E0000112484B714BE81FFF0D085E080938100F7
:107E100082E08093C00088E18093C10086E0809377
:107E2000C20080E18093C4008EE0C9D0259A86E02C
:107E300020E33CEF91E0309385002093840096BBD3
:107E4000B09BFECF1D9AA8958150A9F7CC24DD24C4
:107E500088248394B5E0AB2EA1E19A2EF3E0BF2EE7
:107E6000A2D0813461F49FD0082FAFD0023811F036
:107E7000013811F484E001C083E08DD089C08234E0
:107E800011F484E103C0853419F485E0A6D080C0E4
:107E9000853579F488D0E82EFF2485D0082F10E0AE
:107EA000102F00270E291F29000F111F8ED06801E7
:107EB0006FC0863521F484E090D080E0DECF843638
:107EC00009F040C070D06FD0082F6DD080E0C81688
:107ED00080E7D80618F4F601B7BEE895C0E0D1E017
:107EE00062D089930C17E1F7F0E0CF16F0E7DF06D8
:107EF00018F0F601B7BEE89568D007B600FCFDCFD4
:107F0000A601A0E0B1E02C9130E011968C91119780
:107F100090E0982F8827822B932B1296FA010C0160
:107F200087BEE89511244E5F5F4FF1E0A038BF0790
:107F300051F7F601A7BEE89507B600FCFDCF97BE46
:107F4000E89526C08437B1F42ED02DD0F82E2BD052
:107F50003CD0F601EF2C8F010F5F1F4F84911BD097
:107F6000EA94F801C1F70894C11CD11CFA94CF0C13
:107F7000D11C0EC0853739F428D08EE10CD085E9AC
:107F80000AD08FE07ACF813511F488E018D01DD067
:107F900080E101D065CF982F8091C00085FFFCCF94
:107FA0009093C60008958091C00087FFFCCF809118
:107FB000C00084FD01C0A8958091C6000895E0E648
:107FC000F0E098E1908380830895EDDF803219F02E
:107FD00088E0F5DFFFCF84E1DECF1F93182FE3DFCA
:107FE0001150E9F7F2DF1F91089580E0E8DFEE27F6
:047FF000FF270994CA
:027FFE00040479
:00000001FF
